:1000000035EF2DF0FFFFFFFFE9CFB2F1EACFB3F1FB
:10001000E1CFB4F1E2CFB5F1F2A207D0010E15267F
:10002000000E162217221822F2929EB09E90B2C1A4
:10003000E9FFB3C1EAFFB4C1E1FFB5C1E2FF1100BE
:10004000280E0101E76F6E0EE86F750EE96F6C0EFA
:10005000EA6F6C0EEB6F290EEC6FED6BF56BF66BC8
:10006000F36BF46B0101E2C100F0E3C101F0E4C104
:1000700002F0010EE227000EE323E42300C0F6FFA6
:1000800001C0F7FF02C0F8FF0900F5CF00F000C083
:10009000F0F10052D8B4D6EF11F0F051250A0BE080
:1000A000E0C1E1FFE1C1E2FFF0C1E6FFE04BE12B7F
:1000B000F54BF62BD7D7F16BF26BF36BF46B0101B9
:1000C00028D00101F387010EE227000EE323E42389
:1000D0005ED00101F381010EE227000EE323E42349
:1000E00056D00101F383010EE227000EE323E4233F
:1000F0004ED00101F487010EE227000EE323E42332
:1001000046D00101F385010EE227000EE323E4232C
:100110003ED0E2C1F6FFE3C1F7FFE4C1F8FF0900FA
:10012000F5CF01F2020101512D0ACBE0E2C1F6FF49
:10013000E3C1F7FFE4C1F8FF0900F5CF01F2015177
:10014000200AC7E0E2C1F6FFE3C1F7FFE4C1F8FF10
:100150000900F5CF01F201512B0AC3E0E2C1F6FF1D
:10016000E3C1F7FFE4C1F8FF0900F5CF01F2015147
:10017000230ABFE0E2C1F6FFE3C1F7FFE4C1F8FFE5
:100180000900F5CF01F20151300ABBE002D00201B3
:1001900096D70101F3B3F391F3B7F395E2C1F6FFFC
:1001A000E3C1F7FFE4C1F8FF0900F5CF00F0000E4E
:1001B000016E00C009F20CEC30F0005239E0010190
:1001C000F16BF26BF1C100F0F2C101F00A0E046EA6
:1001D000000E056E39EC2EF0E2C1F6FFE3C1F7FF29
:1001E000E4C1F8FF0900F5CF01F20201015100243A
:1001F0000101F16F000E0120F26F300EF15F000E71
:10020000F25B010EE227000EE323E423E2C1F6FFD6
:10021000E3C1F7FFE4C1F8FF0900F5CF00F0000EDD
:10022000016E00C009F20CEC30F00052CBE137D087
:10023000E2C1F6FFE3C1F7FFE4C1F8FF0900F5CF23
:1002400001F2020101512A0A2AE1E5C1E9FFE6C1F2
:10025000EAFFEECF00F0EECF01F000C0E9FF01C0F1
:10026000EAFFEECFF1F1EECFF2F1E5C1E9FFE6C131
:10027000EAFFEECF00F0EECF01F0020E0026000EF6
:100280000122E5C1E1FFE6C1E2FF00C0E6FF01C0D7
:10029000E6FF010E0101E227000EE323E423010142
:1002A000E2C1F6FFE3C1F7FFE4C1F8FF0900F5CFB3
:1002B00001F2020101512E0AD8A479D0010E0101E8
:1002C000E227000EE323E423E2C1F6FFE3C1F7FFD8
:1002D000E4C1F8FF0900F5CF01F2020101512A0A39
:1002E0002BE1E5C1E9FFE6C1EAFFEECF00F0EECF7A
:1002F00001F000C0E9FF01C0EAFFEECFEEF1EECF62
:10030000EFF1E5C1E9FFE6C1EAFFEECF00F0EECF85
:1003100001F0020E0026000E0122E5C1E1FFE6C158
:10032000E2FF00C0E6FF01C0E6FF010E0101E22787
:10033000000EE323E42339D00101EE6BEF6BE2C141
:10034000F6FFE3C1F7FFE4C1F8FF0900F5CF00F0C5
:10035000000E016E00C009F20CEC30F0005225E0F6
:10036000EEC100F0EFC101F00A0E046E000E056E42
:1003700039EC2EF0E2C1F6FFE3C1F7FFE4C1F8FF6C
:100380000900F5CF01F20201015100240101EE6FD5
:10039000000E0120EF6F300EEE5F000EEF5B010EDE
:1003A000E227000EE323E423CAD7010104D00101B0
:1003B000EE6BEF6BF4890101E2C100F0E3C101F0E3
:1003C000E4C102F0010EE227000EE323E42300C0A3
:1003D000F6FF01C0F7FF02C0F8FF0900F5CFF0F10A
:1003E00000D1F5C100F0F6C101F01200F389E3D7A6
:1003F000F48532D1F38BF4812FD1F4832DD1F38D99
:100400002BD12AD1F38BF38F27D1E5C1E9FFE6C1C8
:10041000EAFFEECF00F0EECF01F000C0E9FF01C02F
:10042000EAFFEECFFDF1EECFFEF1E5C1E9FFE6C157
:10043000EAFFEECF00F0EECF01F0020E0026000E34
:100440000122E5C1E1FFE6C1E2FF00C0E6FF01C015
:10045000E6FF000EFE1902E1000EFD1904E1E70EB1
:10046000FD6F010EFE6F0101FF6B0201006B0101C8
:10047000FF51FD25E96E020100510101FE21EA6EE6
:10048000EECF00F0005204E0FF4B0201002BEFD74B
:1004900002010101EE51EF110CE0020100510101D6
:1004A000EF5D02E1FF51EE5D04E2EEC1FFF1EFC14D
:1004B00000F20101F2510201005D03E10101F1517D
:1004C000FF5D010107E2FF51F15F020100510101EF
:1004D000F25B03D00101F16BF26BF3B716D0F1C1FF
:1004E00000F0F2C101F0010EF15F000EF25B00506E
:1004F00001100BE0E0C1E1FFE1C1E2FF200EE66E7A
:10050000E04BE12BF54BF62BEAD7FFC100F000C220
:1005100001F0010EFF5F000E0201005B00500110B0
:1005200014E0FDC1E9FFFEC1EAFFEECF00F0E0C13B
:10053000E1FFE1C1E2FF00C0E6FF0101E04BE12B7A
:10054000FD4BFE2BF54BF62BE0D70101F3A716D0A0
:10055000F1C100F0F2C101F0010EF15F000EF25B9B
:10056000005001100BE0E0C1E1FFE1C1E2FF200E0D
:10057000E66EE04BE12BF54BF62BEAD773D5E5C1E0
:10058000E9FFE6C1EAFFEECF00F0EECF01F000C0D8
:10059000E9FF01C0EAFFEECFF0F1E5C1E9FFE6C1F6
:1005A000EAFFEECF00F0EECF01F0020E0026000EC3
:1005B0000122E5C1E1FFE6C1E2FF00C0E6FF01C0A4
:1005C000E6FFF00EFD6F010EFE6F010EFF6F000ED5
:1005D0000201006F5DD7C00E0101F313000EF4138A
:1005E0003BD0F051000AD8B4FCD6F0516C0AD8B414
:1005F000FDD6F051660AD8B4FBD6F051450AD8B4FE
:10060000F9D6F051650AD8B4F6D6F051670AD8B4D5
:10061000F4D6F0516F0AD8B4F2D6F051640AD8B4C7
:10062000F0D6F051690AD8B4ECD6F051700AD8B4BB
:10063000E9D6F051580AD8B4E5D6F051780AD8B4C2
:10064000E2D6F051730AD8B4E0D6F051630A97E0CD
:10065000F051750AC0E0B5D70101000EF315006E28
:10066000F451070B016E00500110D8B4CEEF0CF01E
:10067000F4A904D0060EEE6F000EEF6FE5C1E9FF9E
:10068000E6C1EAFFEECF00F0EECF01F000C0E9FFD7
:1006900001C0EAFFEECFF7F1EECFF8F1EECFF9F1BE
:1006A000EECFFAF1E5C1E9FFE6C1EAFFEECF00F0D7
:1006B000EECF01F0040E0026000E0122E5C1E1FF9D
:1006C000E6C1E2FF00C0E6FF01C0E6FF046A056A7A
:1006D000066A076AF7C100F0F8C101F0F9C102F03B
:1006E000FAC103F0BCEC28F0010ED8B0000E006E89
:1006F000005206E00101F97F030EF313000EF4131C
:100700000101FB6BFC6BF7C100F0F8C101F0F9C10E
:1007100002F0FAC103F0046A056A066A076A58EC37
:100720002FF0000ED8A4010E006E0052D8B49DD058
:10073000FAC100F0016A026A036AFF0E00140201A6
:10074000056F000E066F000E06177E0E016F000E7D
:10075000026F036F046F0151055D006E025106596F
:10076000016E00C0FBF101C0FCF1010E005C010153
:10077000FB6F000E0158FC6FFBC100F0FCC101F0E3
:10078000030E046E000E056E39EC2EF000C0FBF176
:1007900001C0FCF10A0E046E000E056E24EC29F077
:1007A00000C0FBF101C0FCF1800E01180201016FD5
:1007B000800E015D02E1000E005C05E2010E010108
:1007C000FB5F000EFC5B0101FB5100080201096F99
:1007D00064EC15F0F7C104F0F8C105F0F9C106F0BA
:1007E000FAC107F041EC27F000C0FDF101C0FEF1B5
:1007F00002C0FFF103C000F2000E046E000E056E91
:10080000000E066E7F0E076EFDC100F0FEC101F006
:10081000FFC102F000C203F0BCEC28F0010ED8B01A
:10082000000E006E005206E0010E0101FB5F000E9B
:10083000FC5B1BD0000E046E000E056E200E066ED3
:10084000820E076EFDC100F0FEC101F0FFC102F093
:1008500000C203F0BCEC28F0000ED8B0010E006E10
:10086000005203E00101FB4BFC2B0101800E006EE6
:10087000800E0101FC19005C02E1FB51000803E35A
:10088000010EF06F03D00101FBC1F0F1F4B11AD0F9
:10089000F4A315D0800EFC19006E7F0E005C02E1FF
:1008A000FC0EFB5D0AE3800EFC19006E800EEF1952
:1008B000005C02E1EE51FB5D02E3010103D00101A6
:1008C000AAEF08F00101EE51EF1106E0F4A304D005
:1008D000010EEE5F000EEF5B000E006EEF51005C4C
:1008E00002E1EE51080803E2080EF06F03D00101A7
:1008F000EEC1F0F1F7C100F0F8C101F0F9C102F06A
:10090000FAC103F0046A056A066A076A58EC2FF018
:10091000000ED8A4010E006E0052D8B465D1FBC100
:1009200009F264EC15F000C004F001C005F002C04B
:1009300006F003C007F0F7C100F0F8C101F0F9C1FB
:1009400002F0FAC103F060EC25F000C0F7F101C03D
:10095000F8F102C0F9F103C0FAF10101F051000809
:100960000201096F64EC15F000C004F001C005F04D
:1009700002C006F003C007F0F7C100F0F8C101F0B3
:10098000F9C102F0FAC103F060EC25F000C001F2F9
:1009900001C002F202C003F203C004F201C2F7F187
:1009A00002C2F8F103C2F9F104C2FAF101C200F087
:1009B00002C201F003C202F004C203F00AEC26F006
:1009C0009DEC2FF000C004F001C005F002C006F05D
:1009D00003C007F001C200F002C201F003C202F03E
:1009E00004C203F04FEC30F0000E046E000E056EF2
:1009F000000E066E7E0E076EBCEC28F0000ED8B01E
:100A0000010E006E00521AE0F7C100F0F8C101F0CB
:100A1000F9C102F0FAC103F0000E046E000E056E7B
:100A2000000E066E7E0E076E69EC18F000C0F7F13E
:100A300001C0F8F102C0F9F103C0FAF1F7C100F00A
:100A4000F8C101F0F9C102F0FAC103F00AEC26F096
:100A500000C005F201C006F202C007F203C008F2AE
:100A60000101F051010F006E016A000E0122020E19
:100A7000046E000E01BEFF0E026E036E04500101F3
:100A800007E000360090013602360336FF0FF7D735
:100A90001C0E0026610E0122000E022200C0F6FF8D
:100AA00001C0F7FF02C0F8FF0900F5CF01F209000D
:100AB000F5CF02F20900F5CF03F20900F5CF04F2F9
:100AC00002010451085D08E10351075D05E102518F
:100AD000065D02E10151055D1EE3F7C100F0F8C1BA
:100AE00001F0F9C102F0FAC103F0CD0E046ECC0E94
:100AF000056E4C0E066E7B0E076E41EC27F000C0B3
:100B0000F7F101C0F8F102C0F9F103C0FAF10101F7
:100B1000FB4BFC2B69D00101F7C100F0F8C101F0DB
:100B2000F9C102F0FAC103F00AEC26F000C005F2A8
:100B300001C006F202C007F203C008F2020E046E02
:100B4000F0C100F0000E016E026E036E0450000151
:100B500007E000360090013602360336FF0FF7D764
:100B60001C0E0026610E0122000E022200C0F6FFBC
:100B700001C0F7FF02C0F8FF0900F5CF01F209003C
:100B8000F5CF02F20900F5CF03F20900F5CF04F228
:100B900002010451085D08E10351075D05E10251BE
:100BA000065D02E10151055D1FE2F7C100F0F8C1E9
:100BB00001F0F9C102F0FAC103F0000E046E000E5C
:100BC000056E200E066E820E076E41EC27F000C007
:100BD000F7F101C0F8F102C0F9F103C0FAF1010E1A
:100BE0000101FB5F000EFC5B01010101F4A39AD03F
:100BF000F4B798D0800E000A006E800EEF19005CEA
:100C000002E1EE510A0804E20A0EEE6F000EEF6FE9
:100C10000101F7C100F0F8C101F0F9C102F0FAC119
:100C200003F00AEC26F000C0FDF101C0FEF102C0A5
:100C3000FFF103C000F20101FD51FE11FF1102019D
:100C4000001144E00A0E046E000E056E066E076E7B
:100C5000FDC100F0FEC101F0FFC102F000C203F0CF
:100C600010EC1CF008C000F009C001F00AC002F04E
:100C70000BC003F0000E0201016F031808E10151DF
:100C8000021805E10151011802E10050000A1EE1BD
:100C9000010E0101EE5F000EEF5B0A0E046E000E06
:100CA000056E066E076EFDC100F0FEC101F0FFC1CA
:100CB00002F000C203F010EC1CF000C0FDF101C016
:100CC000FEF102C0FFF103C000F2B5D7800E0101B2
:100CD000EF19006E800E005C02E1F051EE5D22E241
:100CE000EE51F05D0201096F64EC15F000C004F0F4
:100CF00001C005F002C006F003C007F0F7C100F024
:100D0000F8C101F0F9C102F0FAC103F060EC25F07E
:100D100000C0F7F101C0F8F102C0F9F103C0FAF127
:100D2000EEC1F0F10001050E0101EE25006E000E8E
:100D3000EF21016E0050F15F0150F25BEE51EF11B7
:100D400002E1F4A704D0010EF15F000EF25B030E86
:100D5000F315006EF4C101F0000E011600500110F1
:100D600004E0010EF15F000EF25BF3A54AD0F3A39D
:100D70001AD0010EF315006EF4C101F0000E011639
:100D80000050011003E02D0E006E02D02B0E006EFD
:100D9000E0C1E1FFE1C1E2FF00C0E6FFE04BE12B73
:100DA000F54BF62B14D0010EF315006EF4C101F0D3
:100DB000000E0116005001100AE0E0C1E1FFE1C1A0
:100DC000E2FF200EE66EE04BE12BF54BF62B800E9A
:100DD000006E800EF219005C02E1F15100080FE292
:100DE000E0C1E1FFE1C1E2FF300EE66EE04BE12B36
:100DF000F54BF62B010EF15F000EF25BE8D7010117
:100E00004BD0F3B718D0800E006E800EF219005C44
:100E100002E1F15100080FE2E0C1E1FFE1C1E2FFB0
:100E2000200EE66EE04BE12BF54BF62B010EF15F49
:100E3000000EF25BE8D70101F3A31AD0010EF315FF
:100E4000006EF4C101F0000E01160050011003E025
:100E50002D0E006E02D02B0E006EE0C1E1FFE1C14D
:100E6000E2FF00C0E6FFE04BE12BF54BF62B14D080
:100E7000010EF315006EF4C101F0000E01160050D2
:100E800001100AE0E0C1E1FFE1C1E2FF200EE66EE1
:100E9000E04BE12BF54BF62B0101F7C100F0F8C157
:100EA00001F0F9C102F0FAC103F00AEC26F000C02B
:100EB000FDF101C0FEF102C0FFF103C000F2020E1D
:100EC000046EF0C100F0000E016E026E036E04505D
:100ED000000107E000360090013602360336FF0FAE
:100EE000F7D71C0E0026610E0122000E022200C060
:100EF000F6FF01C0F7FF02C0F8FF0900F5CF04F0CC
:100F00000900F5CF05F00900F5CF06F00900F5CF8F
:100F100007F0FDC100F0FEC101F0FFC102F000C208
:100F200003F010EC1CF0300E0026E0C1E1FFE1C13F
:100F3000E2FF00C0E6FF0101E04BE12BF54BF62B91
:100F4000EE51EF1102E1F4A776D0E0C1E1FFE1C17B
:100F5000E2FF2E0EE66E0101E04BE12BF54BF62B86
:100F6000F051EE5F000EEF5BF05353E0F007020E1E
:100F7000046EF0C100F0000E016E026E036E0450AC
:100F8000010107E000360090013602360336FF0FFC
:100F9000F7D71C0E0026610E0122000E022200C0AF
:100FA000F6FF01C0F7FF02C0F8FF0900F5CF04F01B
:100FB0000900F5CF05F00900F5CF06F00900F5CFDF
:100FC00007F0FDC100F0FEC101F0FFC102F000C258
:100FD00003F010EC1CF00A0E046E000E056E066E97
:100FE000076E10EC1CF008C000F009C001F00AC048
:100FF00002F00BC003F0300E0026E0C1E1FFE1C1BA
:10100000E2FF00C0E6FF0101E04BE12BF54BF62BC0
:10101000ABD7EE51EF110FE0E0C1E1FFE1C1E2FF1C
:10102000300EE66EE04BE12BF54BF62B010EEE5F3A
:10103000000EEF5BEED7F3AB0BD0E0C1E1FFE1C1F7
:10104000E2FF450EE66EE04BE12BF54BF62B0AD0A6
:10105000E0C1E1FFE1C1E2FF650EE66EE04BE12B8E
:10106000F54BF62B800EFC19006E800E005C02E141
:10107000000EFB5D12E2FB510008FB6FFCC1FCF1AE
:10108000E86AFC57E0C1E1FFE1C1E2FF2D0EE66E28
:10109000E04BE12BF54BF62B0BD00101E0C1E1FF5A
:1010A000E1C1E2FF2B0EE66EE04BE12BF54BF62B98
:1010B0000A0E046E000E056EFBC100F0FCC101F0CB
:1010C00024EC29F0300E0026E0C1E1FFE1C1E2FF8F
:1010D00000C0E6FF0101E04BE12BF54BF62B0A0EB9
:1010E000046E000E056EFBC100F0FCC101F024ECA3
:1010F00029F008C000F009C001F0300E0026E0C160
:10110000E1FFE1C1E2FF00C0E6FF0101E04BE12B9E
:10111000F54BF62BF3A71BD0800E006E800EF21954
:10112000005C02E1F151000812E2E0C1E1FFE1C11F
:10113000E2FF200EE66E0101E04BE12BF54BF62BB2
:10114000010EF15F000EF25BF151F211EEE10101CF
:1011500032EF00F00101F4A306D1800EFC19006EFD
:10116000800E005C02E1000EFB5D0AE2010EFB5DF9
:10117000006E000EFC59016E0050EE5F0150EF5BF7
:10118000F7C100F0F8C101F0F9C102F0FAC103F0B3
:101190000AEC26F000C0FDF101C0FEF102C0FFF133
:1011A00003C000F2010E0101F06FF0510A0A3FE0A6
:1011B000020E046EF0C100F0000E016E026E036EAE
:1011C0000450010107E00036009001360236033674
:1011D000FF0FF7D71C0E0026610E0122000E02221F
:1011E00000C0F6FF01C0F7FF02C0F8FF0900F5CF0D
:1011F00001F20900F5CF02F20900F5CF03F2090070
:10120000F5CF04F202010451005D0DE1035101012B
:10121000FF5D09E1020102510101FE5D04E10201ED
:1012200001510101FD5D010102E3F02BBED7010177
:10123000F051EE5D0201056F000E0101EF59020150
:10124000066F05C2EEF106C2EFF1FDC100F0FEC16E
:1012500001F0FFC102F000C203F09DEC2FF000C0CE
:1012600004F001C005F002C006F003C007F0F7C1AA
:1012700000F0F8C101F0F9C102F0FAC103F04FEC3F
:1012800030F000C001F201C002F202C003F203C05C
:1012900004F205C209F264EC15F001C204F002C2C6
:1012A00005F003C206F004C207F041EC27F0000E7F
:1012B000046E000E056E000E066E7E0E076E69EC63
:1012C00018F00AEC26F000C0FDF101C0FEF102C0EA
:1012D000FFF103C000F20101EE51EF1144E00A0EEC
:1012E000046E000E056E066E076EFDC100F0FEC1B5
:1012F00001F0FFC102F000C203F010EC1CF008C0C6
:1013000000F009C001F00AC002F00BC003F0000EAB
:101310000201016F031808E10151021805E10151B2
:10132000011802E10050000A1EE10A0E046E000ED0
:10133000056E066E076EFDC100F0FEC101F0FFC133
:1013400002F000C203F010EC1CF000C0FDF101C07F
:10135000FEF102C0FFF103C000F2010E0101EE5FD9
:10136000000EEF5BB8D70101800E006E800E010108
:10137000EF19005C02E1EE510C0816E3EEC109F230
:101380007DEC1AF0F7C104F0F8C105F0F9C106F0E0
:10139000FAC107F069EC18F000C0F7F101C0F8F1EC
:1013A00002C0F9F103C0FAF1F7C100F0F8C101F091
:1013B000F9C102F0FAC103F0046A056A066A076A15
:1013C00058EC2FF0000ED8A4010E006E0052D8B4D5
:1013D00079D0F7C100F0F8C101F0F9C102F0FAC10B
:1013E00003F00AEC26F0000E0201016F031808E179
:1013F0000151021805E10151011802E10050000AF3
:1014000061E1800E006E800E0101FC19005C02E1BA
:10141000FB51010857E2FBC109F264EC15F000C072
:1014200004F001C005F002C006F003C007F0F7C1E8
:1014300000F0F8C101F0F9C102F0FAC103F060EC6C
:1014400025F05F0E046E700E056E090E066E810E9D
:10145000076EBCEC28F0010ED8B0000E006E0052F2
:1014600006E0090E0101FB5F000EFC5B05D0080ED3
:101470000101FB5F000EFC5BFBC109F264EC15F09F
:1014800000C004F001C005F002C006F003C007F080
:10149000F7C100F0F8C101F0F9C102F0FAC103F0A0
:1014A00060EC25F00AEC26F000C0FDF101C0FEF171
:1014B00002C0FFF103C000F20101F76BF86BF96B9A
:1014C000FA6B39D0F7C100F0F8C101F0F9C102F0B0
:1014D000FAC103F00AEC26F000C0FDF101C0FEF1F4
:1014E00002C0FFF103C000F2FDC100F0FEC101F037
:1014F000FFC102F000C203F09DEC2FF000C004F029
:1015000001C005F002C006F003C007F0F7C100F00B
:10151000F8C101F0F9C102F0FAC103F04FEC30F06C
:1015200000C0F7F101C0F8F102C0F9F103C0FAF10F
:101530000101FB6BFC6B010EF06FF0510A0A3FE0FA
:10154000020E046EF0C100F0000E016E026E036E1A
:101550000450010107E000360090013602360336E0
:10156000FF0FF7D71C0E0026610E0122000E02228B
:1015700000C0F6FF01C0F7FF02C0F8FF0900F5CF79
:1015800001F20900F5CF02F20900F5CF03F20900DC
:10159000F5CF04F202010451005D0DE10351010198
:1015A000FF5D09E1020102510101FE5D04E102015A
:1015B00001510101FD5D010102E3F02BBED70101E4
:1015C000F051EE25006E000EEF21016EFB5100265A
:1015D000FC5101220050F15F0150F25BF4B703D0DF
:1015E000EE51EF1104E0010EF15F000EF25B030E0D
:1015F000F315006EF4C101F0000E01160050011049
:1016000004E0010EF15F000EF25BF3A54AD0F3A3F4
:101610001AD0010EF315006EF4C101F0000E011690
:101620000050011003E02D0E006E02D02B0E006E54
:10163000E0C1E1FFE1C1E2FF00C0E6FFE04BE12BCA
:10164000F54BF62B14D0010EF315006EF4C101F02A
:10165000000E0116005001100AE0E0C1E1FFE1C1F7
:10166000E2FF200EE66EE04BE12BF54BF62B800EF1
:10167000006E800EF219005C02E1F15100080FE2E9
:10168000E0C1E1FFE1C1E2FF300EE66EE04BE12B8D
:10169000F54BF62B010EF15F000EF25BE8D701016E
:1016A0004BD0F3B718D0800E006E800EF219005C9C
:1016B00002E1F15100080FE2E0C1E1FFE1C1E2FF08
:1016C000200EE66EE04BE12BF54BF62B010EF15FA1
:1016D000000EF25BE8D70101F3A31AD0010EF31557
:1016E000006EF4C101F0000E01160050011003E07D
:1016F0002D0E006E02D02B0E006EE0C1E1FFE1C1A5
:10170000E2FF00C0E6FFE04BE12BF54BF62B14D0D7
:10171000010EF315006EF4C101F0000E0116005029
:1017200001100AE0E0C1E1FFE1C1E2FF200EE66E38
:10173000E04BE12BF54BF62B0101F0C100F0F00777
:10174000005252E0020E046EF0C100F0000E016E75
:10175000026E036E0450010107E00036009001366E
:1017600002360336FF0FF7D71C0E0026610E01224A
:10177000000E022200C0F6FF01C0F7FF02C0F8FF12
:101780000900F5CF04F00900F5CF05F00900F5CF09
:1017900006F00900F5CF07F0FDC100F0FEC101F031
:1017A000FFC102F000C203F010EC1CF00A0E046E40
:1017B000000E056E066E076E10EC1CF008C000F0FF
:1017C00009C001F00AC002F00BC003F0300E002681
:1017D000E0C1E1FFE1C1E2FF00C0E6FF0101E04B33
:1017E000E12BF54BF62BA8D7800E006E800EFC196E
:1017F000005C02E1FB5100080FE2E0C1E1FFE1C142
:10180000E2FF300EE66EE04BE12BF54BF62B010EBE
:10181000FB5F000EFC5BE8D70101800E000A006E42
:10182000800EEF19005C02E1EE51080803E2080E99
:10183000F06F03D00101EEC1F0F1F051EE5F000E48
:10184000EF5BF05302E1F4A70AD0E0C1E1FFE1C190
:10185000E2FF2E0EE66EE04BE12BF54BF62BF0C1CE
:1018600009F264EC15F0F7C104F0F8C105F0F9C114
:1018700006F0FAC107F041EC27F0A7EC26F000C013
:10188000FDF101C0FEF102C0FFF103C000F2010151
:10189000F05353E0F007020E046EF0C100F0000EAA
:1018A000016E026E036E0450010107E000360090E5
:1018B000013602360336FF0FF7D71C0E0026610EE5
:1018C0000122000E022200C0F6FF01C0F7FF02C095
:1018D000F8FF0900F5CF04F00900F5CF05F0090085
:1018E000F5CF06F00900F5CF07F0FDC100F0FEC10D
:1018F00001F0FFC102F000C203F010EC1CF00A0E70
:10190000046E000E056E066E076E10EC1CF008C02B
:1019100000F009C001F00AC002F00BC003F0300E65
:101920000026E0C1E1FFE1C1E2FF00C0E6FF0101E6
:10193000E04BE12BF54BF62BAAD7EE51EF110FE060
:10194000E0C1E1FFE1C1E2FF300EE66EE04BE12BCA
:10195000F54BF62B010EEE5F000EEF5BEED7F3A713
:101960001AD0800E006E800EF219005C02E1F15177
:10197000000811E2E0C1E1FFE1C1E2FF200EE66EE6
:10198000E04BE12BF54BF62B010EF15F000EF25B05
:10199000F151F211EFE1010132EF00F0C00EF31549
:1019A0000201016FF4C102F2000E0217000E0219CB
:1019B00002E1000E0119D8A48AD00101F3A929D0AF
:1019C000E5C1E9FFE6C1EAFFEECF00F0EECF01F09E
:1019D00000C0E9FF01C0EAFFEECFFDF1EECFFEF15E
:1019E000EECFFFF1EECF00F2E5C1E9FFE6C1EAFF7D
:1019F000EECF00F0EECF01F0040E0026000E012223
:101A0000E5C1E1FFE6C1E2FF00C0E6FF01C0E6FF7D
:101A100031D0E5C1E9FFE6C1EAFFEECF00F0EECF3D
:101A200001F000C0E9FF01C0EAFFEECFFDF1EECF0B
:101A3000FEF1000EFEBFFF0EFF6F0201006F000EF1
:101A40000101FEBFFF0EFF6F0201006FE5C1E9FF5C
:101A5000E6C1EAFFEECF00F0EECF01F0020E002665
:101A6000000E0122E5C1E1FFE6C1E2FF00C0E6FF92
:101A700001C0E6FF0201800E0019006E800E005CBE
:101A800009E1000E0101FF5D05E1000EFE5D02E1CE
:101A9000000EFD5D010119E2030EF313000EF413B5
:101AA000006A016A026A036AFD51005EFE51015A32
:101AB000FF51025A02010051035A00C0FDF101C05A
:101AC000FEF102C0FFF103C000F2020159D0010192
:101AD000F3A929D0E5C1E9FFE6C1EAFFEECF00F0A6
:101AE000EECF01F000C0E9FF01C0EAFFEECFFDF14B
:101AF000EECFFEF1EECFFFF1EECF00F2E5C1E9FF50
:101B0000E6C1EAFFEECF00F0EECF01F0040E0026B2
:101B1000000E0122E5C1E1FFE6C1E2FF00C0E6FFE1
:101B200001C0E6FF2DD0E5C1E9FFE6C1EAFFEECF37
:101B300000F0EECF01F000C0E9FF01C0EAFFEECFF8
:101B4000FDF1EECFFEF1000EFF6F0201006F000EFF
:101B50000101FF6F0201006FE5C1E9FFE6C1EAFF85
:101B6000EECF00F0EECF01F0020E0026000E0122B3
:101B7000E5C1E1FFE6C1E2FF00C0E6FF01C0E6FF0C
:101B80000201000E0101EF1902E1000EEE1912E14F
:101B9000000E006E0201001909E100500101FF1959
:101BA00005E10050FE1902E1FD51000A010102E1C8
:101BB000EE4BEF2B0101C00EF315006E00C005F2D5
:101BC000D6D001010101010EF06FF0510A0A3FE089
:101BD000020E046EF0C100F0000E016E026E036E84
:101BE0000450010107E0003600900136023603364A
:101BF000FF0FF7D71C0E0026610E0122000E0222F5
:101C000000C0F6FF01C0F7FF02C0F8FF0900F5CFE2
:101C100001F20900F5CF02F20900F5CF03F2090045
:101C2000F5CF04F202010451005D0DE10351010101
:101C3000FF5D09E1020102510101FE5D04E10201C3
:101C400001510101FD5D010102E3F02BBED701014D
:101C50009ED00101010EF06FF051080A3FE0020E24
:101C6000046EF0C100F0000E016E026E036E0450AF
:101C7000010107E000360090013602360336FF0FFF
:101C8000F7D7440E0026610E0122000E022200C08A
:101C9000F6FF01C0F7FF02C0F8FF0900F5CF01F21F
:101CA0000900F5CF02F20900F5CF03F20900F5CFE4
:101CB00004F202010451005D0DE103510101FF5DD9
:101CC00009E1020102510101FE5D04E1020101513D
:101CD0000101FD5D010102E3F02BBED7010157D0E8
:101CE0000101010EF06FF0510C0A3FE0020E046E8C
:101CF000F0C100F0000E016E026E036E045001018F
:101D000007E000360090013602360336FF0FF7D7A2
:101D1000640E0026610E0122000E022200C0F6FFB2
:101D200001C0F7FF02C0F8FF0900F5CF01F209007A
:101D3000F5CF02F20900F5CF03F20900F5CF04F266
:101D400002010451005D0DE103510101FF5D09E154
:101D5000020102510101FE5D04E102010151010194
:101D6000FD5D010102E3F02BBED7010110D002019D
:101D70000551000AD8B425D70551C00AD8B421D7D7
:101D80000551800AD8B465D70551400AA9E0800EF4
:101D9000006E800E0101EF19005C02E1EE51F05D72
:101DA00003E2EEC1F0F10ED00101800EEF19006EDA
:101DB000800E005C02E1F051EE5D04E2F0C1EEF154
:101DC000000EEF6F01010101F151F2110EE0030E5F
:101DD000F315006EF4C101F0000E01160050011061
:101DE00004E0010EF15F000EF25B800EEF19006E51
:101DF000800EF219005C02E1F151EE5D05E2EE5158
:101E0000F15FEF51F25B03D00101F16BF26BC40E95
:101E1000F3150201016F0101F451080B0201026F79
:101E20000251080A02E1400E011909E10101F151D4
:101E3000F21104E0010EF15F000EF25B22D001010D
:101E4000C00EF3150201016F0101F451080B0201EC
:101E5000026F0251080A02E1800E011912E1800EA0
:101E6000006E800E0101F219005C02E1F1510208DE
:101E700005E2020EF15F000EF25B03D00101F16B8F
:101E8000F26B01010101F3A572D0F3A31AD0010E88
:101E9000F315006EF4C101F0000E011600500110A0
:101EA00003E02D0E006E02D02B0E006EE0C1E1FFAC
:101EB000E1C1E2FF00C0E6FFE04BE12BF54BF62B62
:101EC00040D0010EF315006EF4C101F0000E0116B2
:101ED000005001100BE0E0C1E1FFE1C1E2FF200E84
:101EE000E66EE04BE12BF54BF62B2BD0C00EF31535
:101EF0000201016F0101F451080B0201026F02514E
:101F0000080A02E1800E01191CE1E0C1E1FFE1C114
:101F1000E2FF300EE66E0101E04BE12BF54BF62BB4
:101F2000F3AB03D0580E006E02D0780E006EE0C105
:101F3000E1FFE1C1E2FF00C0E6FFE04BE12BF54B22
:101F4000F62B0101F151F21111E0E0C1E1FFE1C115
:101F5000E2FF300EE66EE04BE12BF54BF62B010E67
:101F6000F15F000EF25BF151F211EFE18DD0F15112
:101F7000F21113E0F3B711D0E0C1E1FFE1C1E2FFDC
:101F8000200EE66EE04BE12BF54BF62B010EF15FD8
:101F9000000EF25BF151F211EFE1F3A31AD0010E42
:101FA000F315006EF4C101F0000E0116005001108F
:101FB00003E02D0E006E02D02B0E006EE0C1E1FF9B
:101FC000E1C1E2FF00C0E6FFE04BE12BF54BF62B51
:101FD00014D0010EF315006EF4C101F0000E0116CD
:101FE000005001100AE0E0C1E1FFE1C1E2FF200E74
:101FF000E66EE04BE12BF54BF62BC00EF31502011C
:10200000016F0101F451080B0201026F0251080A2D
:1020100002E1400E01190CE1E0C1E1FFE1C1E2FF84
:10202000300EE66E0101E04BE12BF54BF62B2CD088
:102030000101C00EF3150201016F0101F451080BFB
:102040000201026F0251080A02E1800E01191CE12F
:10205000E0C1E1FFE1C1E2FF300EE66E0101E04BBD
:10206000E12BF54BF62BF3AB03D0580E006E02D0EC
:10207000780E006EE0C1E1FFE1C1E2FF00C0E6FFC3
:10208000E04BE12BF54BF62B01010101800E006EB8
:10209000800EEF19005C02E1EE51F05D0BE2E0C151
:1020A000E1FFE1C1E2FF300EE66EE04BE12BF54BC4
:1020B000F62BEAD70101EEC100F0EFC101F0010EED
:1020C000EE5F000EEF5B00500110D8B450D1C00E8F
:1020D000F315006E00C001F22ED101010101020EC4
:1020E000046EEEC100F0EFC101F0000EEFBFFF0E75
:1020F000026E036E0450010107E0003600900136C5
:1021000002360336FF0FF7D71C0E0026610E0122A0
:10211000000E022200C0F6FF01C0F7FF02C0F8FF68
:102120000900F5CF04F00900F5CF05F00900F5CF5F
:1021300006F00900F5CF07F0FDC100F0FEC101F087
:10214000FFC102F000C203F010EC1CF00A0E046E96
:10215000000E056E066E076E10EC1CF008C000F055
:1021600009C001F00AC002F00BC003F0300E0024D9
:102170000101F06FF0D00101F3AB4ED0020E046EFE
:10218000EEC100F0EFC101F0000EEFBFFF0E026ED6
:10219000036E0450010107E000360090013602365C
:1021A0000336FF0FF7D70101440E0026610E01220E
:1021B000000E022200C0F6FF01C0F7FF02C0F8FFC8
:1021C0000900F5CF04F00900F5CF05F00900F5CFBF
:1021D00006F00900F5CF07F0FDC100F0FEC101F0E7
:1021E000FFC102F000C203F010EC1CF00F0E00164D
:1021F000000E011602160316940E0026610E01222F
:10220000000E022200C0F6FF01C0F7FF02C0F8FF77
:102210000900F5CFF0F14ED0020E046EEEC100F0D1
:10222000EFC101F0000E0101EFBFFF0E026E036E61
:102230000450010107E000360090013602360336F3
:10224000FF0FF7D70101440E0026610E0122000E98
:10225000022200C0F6FF01C0F7FF02C0F8FF09002C
:10226000F5CF04F00900F5CF05F00900F5CF06F031
:102270000900F5CF07F0FDC100F0FEC101F0FFC17C
:1022800002F000C203F010EC1CF00F0E0016000E5E
:10229000011602160316A60E0026610E0122000E7C
:1022A000022200C0F6FF01C0F7FF02C0F8FF0900DC
:1022B000F5CFF0F100014FD0020E046EEEC100F038
:1022C000EFC101F0000E0101EFBFFF0E026E036EC1
:1022D0000450010107E00036009001360236033653
:1022E000FF0FF7D7640E0026610E0122000E0222B6
:1022F00000C0F6FF01C0F7FF02C0F8FF0900F5CFEC
:1023000004F00900F5CF05F00900F5CF06F009004B
:10231000F5CF07F0FDC100F0FEC101F0FFC102F0F2
:1023200000C203F010EC1CF0070E00140101F06F66
:10233000300EF02710D002010151000AD8B4CDD6DA
:102340000151C00AD8B4C9D60151800AD8B413D7F4
:102350000151400AB1E0E0C1E1FFE1C1E2FFF0C19B
:10236000E6FF0101E04BE12BF54BF62BA3D6F3A7DB
:102370001AD0800E006E800EF219005C02E1F1515D
:10238000000811E2E0C1E1FFE1C1E2FF200EE66ECC
:10239000E04BE12BF54BF62B010EF15F000EF25BEB
:1023A000F151F211EFE1010132EF00F0F5C100F05F
:1023B000F6C101F0120001017A6B5DC100F05EC14F
:1023C00001F05FC102F060C103F09DEC2FF0FB0E45
:1023D000046E5C0E056E1D0E066E6B0E076E41ECF4
:1023E00027F000C0B6F101C0B7F102C0B8F103C0D8
:1023F000B9F1B6C1A2F1B7C1A3F1B8C1A4F1B9C195
:10240000A5F161C100F062C101F063C102F064C1D5
:1024100003F09DEC2FF0FB0E046E5C0E056E1D0E9E
:10242000066E6B0E076E41EC27F000C0C2F101C0D2
:10243000C3F102C0C4F103C0C5F1C2C1A6F1C3C15A
:10244000A7F1C4C1A8F1C5C1A9F165C100F066C179
:1024500001F067C102F068C103F09DEC2FF0FB0EA4
:10246000046E5C0E056E1D0E066E6B0E076E41EC63
:1024700027F000C0BEF101C0BFF102C0C0F103C02F
:10248000C1F1BEC1AAF1BFC1ABF1C0C1ACF1C1C1C4
:10249000ADF169C100F06AC101F06BC102F06CC11D
:1024A00003F09DEC2FF0FB0E046E5C0E056E1D0E0E
:1024B000066E6B0E076E41EC27F000C0BAF101C04A
:1024C000BBF102C0BCF103C0BDF1BAC1AEF1BBC1EA
:1024D000AFF1BCC1B0F1BDC1B1F1170E046EB70EC2
:1024E000056E510E066E710E076EB6C100F0B7C1D3
:1024F00001F0B8C102F0B9C103F04FEC30F000C0F8
:10250000B6F101C0B7F102C0B8F103C0B9F1B6C16C
:10251000A2F1B7C1A3F1B8C1A4F1B9C1A5F1170ED9
:10252000046EB70E056E510E066E710E076EC2C1B7
:1025300000F0C3C101F0C4C102F0C5C103F04FEC0B
:1025400030F000C0C2F101C0C3F102C0C4F103C049
:10255000C5F1C2C1A6F1C3C1A7F1C4C1A8F1C5C1EB
:10256000A9F1170E046EB70E056E510E066E710EB0
:10257000076EBEC100F0BFC101F0C0C102F0C1C111
:1025800003F04FEC30F000C0BEF101C0BFF102C05B
:10259000C0F103C0C1F1BEC1AAF1BFC1ABF1C0C15E
:1025A000ACF1C1C1ADF1170E046EB70E056E510E40
:1025B000066E710E076EBAC100F0BBC101F0BCC15E
:1025C00002F0BDC103F04FEC30F000C0BAF101C021
:1025D000BBF102C0BCF103C0BDF1BAC1AEF1BBC1D9
:1025E000AFF1BCC1B0F1BDC1B1F1B6C100F0B7C12E
:1025F00001F0B8C102F0B9C103F09A0E046E690E81
:10260000056E230E066E8A0E076E41EC27F0000E53
:10261000046E800E056E940E066E870E076E69ECD2
:1026200018F000C0B6F101C0B7F102C0B8F103C0A4
:10263000B9F1B6C1A2F1B7C1A3F1B8C1A4F1B9C152
:10264000A5F1C2C100F0C3C101F0C4C102F0C5C10F
:1026500003F09A0E046E690E056E230E066E8A0E46
:10266000076E41EC27F0000E046E800E056E940E8E
:10267000066E870E076E69EC18F000C0A6F101C067
:10268000A7F102C0A8F103C0A9F1BEC100F0BFC10B
:1026900001F0C0C102F0C1C103F09A0E046E690ED0
:1026A000056E230E066E8A0E076E41EC27F0000EB3
:1026B000046E800E056E940E066E870E076E69EC32
:1026C00018F000C0AAF101C0ABF102C0ACF103C028
:1026D000ADF1BAC100F0BBC101F0BCC102F0BDC197
:1026E00003F09A0E046E690E056E230E066E8A0EB6
:1026F000076E41EC27F0000E046E800E056E940EFE
:10270000066E870E076E69EC18F000C0AEF101C0CE
:10271000AFF102C0B0F103C0B1F1B6C104F0B7C16E
:1027200005F0B8C106F0B9C107F0000E006E000E4A
:10273000016E480E026E850E036EBCEC28F0010E91
:10274000D8B0000E006E005209E0CD0E0101A26F5C
:10275000CC0EA36F470EA46F850EA56FA6C104F023
:10276000A7C105F0A8C106F0A9C107F0000E006ED0
:10277000000E016E480E026E850E036EBCEC28F052
:10278000010ED8B0000E006E005209E0CD0E01011E
:10279000A66FCC0EA76F470EA86F850EA96FAAC1B2
:1027A00004F0ABC105F0ACC106F0ADC107F0000EFE
:1027B000006E000E016E480E026E850E036EBCECBC
:1027C00028F0010ED8B0000E006E005209E0CD0EC8
:1027D0000101AA6FCC0EAB6F470EAC6F850EAD6FCB
:1027E000AEC104F0AFC105F0B0C106F0B1C107F051
:1027F000000E006E000E016E480E026E850E036E16
:10280000BCEC28F0010ED8B0000E006E005209E0BA
:10281000CD0E0101AE6FCC0EAF6F470EB06F850EBF
:10282000B16F000E296E000E2A6E000E2B6E7F0E09
:102830002C6EAFC000F0000E0001AFBFFF0E016EA6
:1028400036EC2FF000C029F001C02AF002C02BF0B6
:1028500003C02CF0000E046E000E056E200E066EF6
:10286000820E076E60EC25F0A2C104F0A3C105F052
:10287000A4C106F0A5C107F069EC18F000C0B6F1DC
:1028800001C0B7F102C0B8F103C0B9F1B6C1A2F1FD
:10289000B7C1A3F1B8C1A4F1B9C1A5F1000E296E69
:1028A000000E2A6E000E2B6E7F0E2C6EB0C000F054
:1028B000000EB0BFFF0E016E36EC2FF000C029F005
:1028C00001C02AF002C02BF003C02CF0000E046EF1
:1028D000000E056E200E066E820E076E60EC25F06F
:1028E000A6C104F0A7C105F0A8C106F0A9C107F070
:1028F00069EC18F000C0A6F101C0A7F102C0A8F170
:1029000003C0A9F1000E296E000E2A6E000E2B6E78
:102910007F0E2C6EB1C000F0000EB1BFFF0E016E35
:1029200036EC2FF000C029F001C02AF002C02BF0D5
:1029300003C02CF0000E046E000E056E200E066E15
:10294000820E076E60EC25F0AAC104F0ABC105F061
:10295000ACC106F0ADC107F069EC18F000C0AAF1F7
:1029600001C0ABF102C0ACF103C0ADF1000E296EA5
:10297000000E2A6E000E2B6E7F0E2C6EB2C000F081
:10298000000EB2BFFF0E016E36EC2FF000C029F032
:1029900001C02AF002C02BF003C02CF0000E046E20
:1029A000000E056E200E066E820E076E60EC25F09E
:1029B000AEC104F0AFC105F0B0C106F0B1C107F07F
:1029C00069EC18F000C0AEF101C0AFF102C0B0F187
:1029D00003C0B1F12F0E0101D16F000ED26F480E6E
:1029E000D36F620ED46F000ED56FB6C1D6F1B7C1EA
:1029F000D7F1B8C1D8F1B9C1D9F1C7EC2EF0010EA9
:102A0000D16F010ED26F2F0ED36F000ED46F7EECFC
:102A10002DF02F0ED16F000ED26F500ED36F620EBD
:102A2000D46F000ED56FAAC1D6F1ABC1D7F1ACC13E
:102A3000D8F1ADC1D9F1C7EC2EF0010ED16F090E5E
:102A4000D26F2F0ED36F000ED46F7EEC2DF02F0EB1
:102A5000D16F000ED26F580ED36F620ED46F000E7E
:102A6000D56FA6C1D6F1A7C1D7F1A8C1D8F1A9C128
:102A7000D9F1C7EC2EF0020ED16F010ED26F2F0EDE
:102A8000D36F000ED46F7EEC2DF02F0ED16F000EA1
:102A9000D26F600ED36F620ED46F000ED56FAEC1D1
:102AA000D6F1AFC1D7F1B0C1D8F1B1C1D9F1C7ECFE
:102AB0002EF0020ED16F090ED26F2F0ED36F000EC3
:102AC000D46F7EEC2DF01200800E02010919006E09
:102AD000800E000A005CD8B081D109510008046E54
:102AE00004C009F2800E0418006E800E6E0A005CAD
:102AF000D8A0C6D0640E046E09C200F0EBEC29F039
:102B0000120E0026000E00BEFF0E016E000E012206
:102B1000020E046E000E01BEFF0E026E036E045024
:102B2000000107E000360090013602360336FF0F41
:102B3000F7D70001B40E0026600E0122000E02221B
:102B400000C0F6FF01C0F7FF02C0F8FF0900F5CF93
:102B50000AF20900F5CF0BF20900F5CF0CF20900DB
:102B6000F5CF0DF2640E046E09C200F0EBEC29F013
:102B700008C000F00A0E046EEBEC29F0090E0026E6
:102B8000000E00BEFF0E016E000E0122020E046E4A
:102B9000000E01BEFF0E026E036E0450000107E03E
:102BA00000360090013602360336FF0FF7D70001DA
:102BB000B40E0026600E0122000E022200C0F6FFB5
:102BC00001C0F7FF02C0F8FF0900F5CF00F00900CF
:102BD000F5CF01F00900F5CF02F00900F5CF03F0C1
:102BE0000AC204F00BC205F00CC206F00DC207F0D9
:102BF00041EC27F000C00AF201C00BF202C00CF257
:102C000003C00DF20A0E046E09C200F0EBEC29F0CD
:102C100008C000F0020E046E000E00BEFF0E016E32
:102C2000026E036E0450000107E00036009001368A
:102C300002360336FF0FF7D70001B40E0026600EF0
:102C40000122000E022200C0F6FF01C0F7FF02C001
:102C5000F8FF0900F5CF00F00900F5CF01F00900F9
:102C6000F5CF02F00900F5CF03F00AC204F00BC261
:102C700005F00CC206F00DC207F041EC27F012007F
:102C8000800E0A0A006E800E02010919005C76E2CD
:102C90000A0E046E09C200F0EBEC29F0090E0026C2
:102CA000000E00BEFF0E016E000E0122020E046E29
:102CB000000E01BEFF0E026E036E0450000107E01D
:102CC00000360090013602360336FF0FF7D70001B9
:102CD000B40E0026600E0122000E022200C0F6FF94
:102CE00001C0F7FF02C0F8FF0900F5CF0AF20900A2
:102CF000F5CF0BF20900F5CF0CF20900F5CF0DF27C
:102D00000A0E046E09C200F0EBEC29F008C000F0D6
:102D1000020E046E000E00BEFF0E016E026E036E08
:102D20000450000107E000360090013602360336F9
:102D3000FF0FF7D70001B40E0026600E0122000E2F
:102D4000022200C0F6FF01C0F7FF02C0F8FF090031
:102D5000F5CF00F00900F5CF01F00900F5CF02F042
:102D60000900F5CF03F00AC204F00BC205F00CC253
:102D700006F00DC207F041EC27F012000001020E30
:102D8000046E09C200F0000E020109BFFF0E016EC1
:102D9000026E036E0450020107E000360090013617
:102DA00002360336FF0FF7D70201B40E0026600E7D
:102DB0000122000E022200C0F6FF01C0F7FF02C090
:102DC000F8FF0900F5CF00F00900F5CF01F0090088
:102DD000F5CF02F00900F5CF03F01200800E0919BB
:102DE000006E800E6E0A005CD8A0C6D0640E046E21
:102DF00009C200F0EBEC29F0120E0026000E00BE16
:102E0000FF0E016E000E0122020E046E000E01BEC6
:102E1000FF0E026E036E0450000107E000360090C2
:102E2000013602360336FF0FF7D70001E80E002601
:102E3000600E0122000E022200C0F6FF01C0F7FF63
:102E400002C0F8FF0900F5CF0AF20900F5CF0BF236
:102E50000900F5CF0CF20900F5CF0DF2640E046EF7
:102E600009C200F0EBEC29F008C000F00A0E046E75
:102E7000EBEC29F0090E0026000E00BEFF0E016EDD
:102E8000000E0122020E046E000E01BEFF0E026E45
:102E9000036E0450000107E0003600900136023650
:102EA0000336FF0FF7D70001E80E0026600E01225F
:102EB000000E022200C0F6FF01C0F7FF02C0F8FFBB
:102EC0000900F5CF00F00900F5CF01F00900F5CFBA
:102ED00002F00900F5CF03F00AC204F00BC205F0BE
:102EE0000CC206F00DC207F041EC27F000C00AF258
:102EF00001C00BF202C00CF203C00DF20A0E046E08
:102F000009C200F0EBEC29F008C000F0020E046EDC
:102F1000000E00BEFF0E016E026E036E0450000133
:102F200007E000360090013602360336FF0FF7D770
:102F30000001E80E0026600E0122000E022200C0F1
:102F4000F6FF01C0F7FF02C0F8FF0900F5CF00F05F
:102F50000900F5CF01F00900F5CF02F00900F5CF27
:102F600003F00AC204F00BC205F00CC206F00DC259
:102F700007F041EC27F01200800E0A0A006E800E66
:102F800002010919005C76E20A0E046E09C200F023
:102F9000EBEC29F0090E0026000E00BEFF0E016EBC
:102FA000000E0122020E046E000E01BEFF0E026E24
:102FB000036E0450000107E000360090013602362F
:102FC0000336FF0FF7D70001E80E0026600E01223E
:102FD000000E022200C0F6FF01C0F7FF02C0F8FF9A
:102FE0000900F5CF0AF20900F5CF0BF20900F5CF81
:102FF0000CF20900F5CF0DF20A0E046E09C200F0C2
:10300000EBEC29F008C000F0020E046E000E00BECA
:10301000FF0E016E026E036E0450000107E00036E1
:103020000090013602360336FF0FF7D70001E80E95
:103030000026600E0122000E022200C0F6FF01C031
:10304000F7FF02C0F8FF0900F5CF00F00900F5CF47
:1030500001F00900F5CF02F00900F5CF03F00AC234
:1030600004F00BC205F00CC206F00DC207F041ECF3
:1030700027F012000001020E046E09C200F0000EDB
:10308000020109BFFF0E016E026E036E04500201C1
:1030900007E000360090013602360336FF0FF7D7FF
:1030A000E80E0026600E0122000E022200C0F6FF8C
:1030B00001C0F7FF02C0F8FF0900F5CF00F00900DA
:1030C000F5CF01F00900F5CF02F00900F5CF03F0CC
:1030D00012000001025006180E6E086A096A0B6A97
:1030E000035007645DEF19F006500A6E068E028EDB
:1030F00003500B6E0750036E000E0B64ADEF18F01B
:103100000B50075ED8B44EEF19F0070E07641CEFA2
:1031100019F0075E00C008F001C000F002C001F025
:10312000026A074E4EEF19F00764F1EF18F0075EE0
:1031300000C008F001C000F0016A074E4EEF19F020
:103140000764CFEF18F0075E00C008F0006A074E72
:103150004EEF19F00764B6EF18F00AC002F005C090
:1031600001F004C000F0086A7AEF1AF0030E076459
:10317000C1EF18F0075E08380F0B086E074E4EEFD0
:1031800019F0D8900832074E4EEF19F0D890083257
:10319000074E4EEF19F0D89008324EEF19F0030E9B
:1031A0000764E0EF18F0075E08380F0B086E003870
:1031B000F00B082600380F0B006E074E4EEF19F08B
:1031C000D89000320832074E4EEF19F0D8900032F6
:1031D0000832074E4EEF19F0D890003208324EEF09
:1031E00019F0030E076408EF19F0075E08380F0B9B
:1031F000086E0038F00B082600380F0B006E0138FF
:10320000F00B002601380F0B016E074E4EEF19F040
:10321000D890013200320832074E4EEF19F0D890A4
:10322000013200320832074E4EEF19F0D8900132C9
:10323000003208324EEF19F0030E076439EF19F02F
:10324000075E08380F0B086E0038F00B08260038B0
:103250000F0B006E0138F00B002601380F0B016ECA
:103260000238F00B012602380F0B026E074E4EEFAC
:1032700019F0D8900232013200320832074E4EEF78
:1032800019F0D8900232013200320832074E4EEF68
:1032900019F0D8900232013200320832096A000E69
:1032A0000EAE42EF1AF0081E001E011E021E082A72
:1032B00000220122022242EF1AF00750D8A463EF45
:1032C00019F07AEF1AF0096A02C00AF0028E068E2F
:1032D0000750035C076ED8B435EF1AF0070E076489
:1032E00003EF1AF0075E0450096E0550046E065095
:1032F000056E066A074E35EF1AF0070E0764D8EF21
:1033000019F0075E0450096E0550046E056A074EF9
:1033100035EF1AF0070E0764B6EF19F0075E045098
:10332000096E046A074E35EF1AF0070E07649DEF29
:1033300019F00AC002F07AEF1AF0030E0764A8EF42
:1033400019F0075E09380F0B096E074E35EF1AF0BA
:10335000D8900932074E35EF1AF0D8900932074E4F
:1033600035EF1AF0D890093235EF1AF0030E0764E2
:10337000C7EF19F0075E09380F0B096E0438F00B20
:10338000092604380F0B046E074E35EF1AF0D8905B
:1033900004320932074E35EF1AF0D8900432093260
:1033A000074E35EF1AF0D8900432093235EF1AF093
:1033B000030E0764EFEF19F0075E09380F0B096E73
:1033C0000438F00B092604380F0B046E0538F00B97
:1033D000042605380F0B056E074E35EF1AF0D8900E
:1033E000053204320932074E35EF1AF0D890053213
:1033F00004320932074E35EF1AF0D8900532043204
:10340000093235EF1AF0030E076420EF1AF0075E59
:1034100009380F0B096E0438F00B092604380F0B1E
:10342000046E0538F00B042605380F0B056E0638C0
:10343000F00B052606380F0B066E074E35EF1AF017
:10344000D8900632053204320932074E35EF1AF0B1
:10345000D8900632053204320932074E35EF1AF0A1
:10346000D8900632053204320932086A000E0EAED8
:1034700042EF1AF0091E041E051E061E092A042228
:103480000522062209500826045000220550012278
:10349000065002220EBE59EF1AF0D8A068EF1AF0BB
:1034A0000232013200320832033E68EF1AF074EF44
:1034B0001AF0D8B06EEF1AF0000E081E001E011EA2
:1034C000021E082A0022012202220A7E6EEF1AF052
:1034D000010E0C6EE2EC22F07CEF1AF0020E0C6E84
:1034E000E2EC22F07CEF1AF0040E0C6EFFEC2FF0F1
:1034F0007CEF1AF0000E0C6E12006E0E0201095DD8
:10350000D8A0D0D0640E046E09C200F0B1EC2FF048
:10351000120E0026016A000E0122020E046E000E39
:1035200001BEFF0E026E036E0450000107E000367C
:103530000090013602360336FF0FF7D70001B40EB4
:103540000026600E0122000E022200C0F6FF01C01C
:10355000F7FF02C0F8FF0900F5CF00F00900F5CF32
:1035600001F00900F5CF02F00900F5CF03F0000EDD
:10357000046E000E056E000E066E7E0E076E41ECA8
:1035800027F000C00AF201C00BF202C00CF203C027
:103590000DF2640E046E09C200F0B1EC2FF008C009
:1035A00000F00A0E046EB1EC2FF0090E0026016A3D
:1035B000000E0122020E046E000E01BEFF0E026E0E
:1035C000036E0450000107E0003600900136023619
:1035D0000336FF0FF7D70001B40E0026600E01225C
:1035E000000E022200C0F6FF01C0F7FF02C0F8FF84
:1035F0000900F5CF00F00900F5CF01F00900F5CF83
:1036000002F00900F5CF03F00AC204F00BC205F086
:103610000CC206F00DC207F041EC27F000C00AF220
:1036200001C00BF202C00CF203C00DF20A0E046ED0
:1036300009C200F0B1EC2FF008C000F0020E046ED9
:10364000000E016E026E036E0450000107E00036AA
:103650000090013602360336FF0FF7D70001B40E93
:103660000026600E0122000E022200C0F6FF01C0FB
:10367000F7FF02C0F8FF0900F5CF00F00900F5CF11
:1036800001F00900F5CF02F00900F5CF03F00AC2FE
:1036900004F00BC205F00CC206F00DC207F041ECBD
:1036A00027F01200020109510A08D8B083D00A0E8F
:1036B000046E09C200F0B1EC2FF0090E0026016A79
:1036C000000E0122020E046E000E01BEFF0E026EFD
:1036D000036E0450000107E0003600900136023608
:1036E0000336FF0FF7D70001B40E0026600E01224B
:1036F000000E022200C0F6FF01C0F7FF02C0F8FF73
:103700000900F5CF00F00900F5CF01F00900F5CF71
:1037100002F00900F5CF03F0000E046E000E056EF6
:10372000000E066E7E0E076E41EC27F000C00AF216
:1037300001C00BF202C00CF203C00DF20A0E046EBF
:1037400009C200F0B1EC2FF008C000F0020E046EC8
:10375000000E016E026E036E0450000107E0003699
:103760000090013602360336FF0FF7D70001B40E82
:103770000026600E0122000E022200C0F6FF01C0EA
:10378000F7FF02C0F8FF0900F5CF00F00900F5CF00
:1037900001F00900F5CF02F00900F5CF03F00AC2ED
:1037A00004F00BC205F00CC206F00DC207F041ECAC
:1037B00027F012000001020E046E09C200F0000E94
:1037C000016E026E036E0450000107E000360090A7
:1037D000013602360336FF0FF7D7B40E0026600E0F
:1037E0000122000E022200C0F6FF01C0F7FF02C056
:1037F000F8FF0900F5CF00F00900F5CF01F009004E
:10380000F5CF02F00900F5CF03F0000E046E000EB4
:10381000056E000E066E7E0E076E41EC27F012005C
:1038200000010B6A0A6A096A086A0E6A03340836DC
:103830000450085E0550D8A0053C095E0650D8A08B
:10384000063C0A5E0750D8A0073C0B5EE86AD8A089
:10385000010E0E5E0336070E0C6E03340836093671
:103860000A360B360E36045003A04AEF1CF0085EF1
:103870000550D8A0053C095E0650D8A0063C0A5E5B
:103880000750D8A0073C0B5EE86AD8A0010E0E5E78
:103890005BEF1CF008260550D8B0053C0926065001
:1038A000D8B0063C0A260750D8B0073C0B26E86A79
:1038B000D8B0010E0E2603360C2E2DEF1CF002346C
:1038C000083609360A360B360E36045003A07CEF54
:1038D0001CF0085E0550D8A0053C095E0650D8A033
:1038E000063C0A5E0750D8A0073C0B5EE86AD8A0E9
:1038F000010E0E5E8DEF1CF008260550D8B0053C79
:1039000009260650D8B0063C0A260750D8B0073C16
:103910000B26E86AD8B0010E0E260236070E0C6E92
:103920000234083609360A360B360E36045002A029
:10393000ADEF1CF0085E0550D8A0053C095E0650AE
:10394000D8A0063C0A5E0750D8A0073C0B5EE86A88
:10395000D8A0010E0E5EBEEF1CF008260550D8B0B0
:10396000053C09260650D8B0063C0A260750D8B0B8
:10397000073C0B26E86AD8B0010E0E2602360C2E44
:1039800090EF1CF00134083609360A360B360E3635
:10399000045002A0DFEF1CF0085E0550D8A0053CE3
:1039A000095E0650D8A0063C0A5E0750D8A0073C26
:1039B0000B5EE86AD8A0010E0E5EF0EF1CF0082640
:1039C0000550D8B0053C09260650D8B0063C0A265A
:1039D0000750D8B0073C0B26E86AD8B0010E0E2677
:1039E0000136070E0C6E0134083609360A360B36DE
:1039F0000E36045001A010EF1DF0085E0550D8A04F
:103A0000053C095E0650D8A0063C0A5E0750D8A0C7
:103A1000073C0B5EE86AD8A0010E0E5E21EF1DF098
:103A200008260550D8B0053C09260650D8B0063CFB
:103A30000A260750D8B0073C0B26E86AD8B0010E1A
:103A40000E2601360C2EF3EF1CF000340836093632
:103A50000A360B360E36045001A042EF1DF0085E08
:103A60000550D8A0053C095E0650D8A0063C0A5E69
:103A70000750D8A0073C0B5EE86AD8A0010E0E5E86
:103A800053EF1DF008260550D8B0053C0926065016
:103A9000D8B0063C0A260750D8B0073C0B26E86A87
:103AA000D8B0010E0E260036070E0C6E0034083614
:103AB00009360A360B360E36045000A073EF1DF09F
:103AC000085E0550D8A0053C095E0650D8A0063C0B
:103AD0000A5E0750D8A0073C0B5EE86AD8A0010E2A
:103AE0000E5E84EF1DF008260550D8B0053C09266F
:103AF0000650D8B0063C0A260750D8B0073C0B2623
:103B0000E86AD8B0010E0E2600360C2E56EF1DF0D6
:103B100000B099EF1DF0045008260550D8B0053CC0
:103B200009260650D8B0063C0A260750D8B0073CF4
:103B30000B261200000E296E000E2A6E000E2B6E50
:103B40007F0E2C6E38D10001AF51010F006E00C006
:103B5000AFF0050E0101D16F000ED26F00C0D3F19E
:103B600087EC2FF0AFC000F0000E0001AFBFFF0EDA
:103B7000016E36EC2FF029C004F02AC005F02BC0EE
:103B800006F02CC007F041EC27F000C029F001C07E
:103B90002AF002C02BF003C02CF02F0E0101D16FD0
:103BA000000ED26FE80ED36F610ED46F000ED56F8A
:103BB0002DC0D6F12EC0D7F1000E046E000E056E9A
:103BC000200E066E820E076E60EC25F000C0D8F164
:103BD00001C0D9F102C0DAF103C0DBF1C7EC2EF06D
:103BE0000AD10001B051010F006E00C0B0F0060E06
:103BF0000101D16F000ED26F00C0D3F187EC2FF01E
:103C0000B0C000F0000E0001B0BFFF0E016E36EC38
:103C10002FF029C004F02AC005F02BC006F02CC0FC
:103C200007F041EC27F000C029F001C02AF002C0E3
:103C30002BF003C02CF02F0E0101D16F000ED26FBC
:103C4000F40ED36F610ED46F000ED56F2DC0D6F178
:103C50002EC0D7F1000E046E000E056E200E066E0B
:103C6000820E076E60EC25F000C0D8F101C0D9F1DA
:103C700002C0DAF103C0DBF1C7EC2EF0BCD00001CA
:103C8000B151010F006E00C0B1F0070E0101D16FFC
:103C9000000ED26F00C0D3F187EC2FF0B1C000F05E
:103CA000000E0001B1BFFF0E016E36EC2FF029C0EF
:103CB00004F02AC005F02BC006F02CC007F041EC40
:103CC00027F000C029F001C02AF002C02BF003C089
:103CD0002CF02F0E0101D16F000ED26F000ED36FAA
:103CE000620ED46F000ED56F2DC0D6F12EC0D7F165
:103CF000000E046E000E056E200E066E820E076E1C
:103D000060EC25F000C0D8F101C0D9F102C0DAF1B1
:103D100003C0DBF1C7EC2EF06ED00001B251010FF1
:103D2000006E00C0B2F0080E0101D16F000ED26F1C
:103D300000C0D3F187EC2FF0B2C000F0000E0001FC
:103D4000B2BFFF0E016E36EC2FF029C004F02AC07E
:103D500005F02BC006F02CC007F041EC27F000C0A6
:103D600029F001C02AF002C02BF003C02CF02F0E66
:103D70000101D16F000ED26F0C0ED36F620ED46FA3
:103D8000000ED56F2DC0D6F12EC0D7F1000E046EF7
:103D9000000E056E200E066E820E076E60EC25F09A
:103DA00000C0D8F101C0D9F102C0DAF103C0DBF1E3
:103DB000C7EC2EF020D00101000E2E1802E1010EFA
:103DC0002D180101D8B4BFD6000E2E1802E1020E44
:103DD0002D180101D8B405D7000E2E1802E1030EEC
:103DE0002D180101D8B44BD7000E2E1802E1040E95
:103DF0002D18010192E0020E0101D16F010ED26F68
:103E00002F0ED36F000ED46F7EEC2DF01200000E3B
:103E1000296E000E2A6E000E2B6E7F0E2C6E34D192
:103E20000001AF05006E00C0AFF0050E0101D16FBB
:103E3000000ED26F00C0D3F187EC2FF0AFC000F0BE
:103E4000000E0001AFBFFF0E016E36EC2FF029C04F
:103E500004F02AC005F02BC006F02CC007F041EC9E
:103E600027F000C029F001C02AF002C02BF003C0E7
:103E70002CF02F0E0101D16F000ED26F180ED36FF0
:103E8000620ED46F000ED56F2DC0D6F12EC0D7F1C3
:103E9000000E046E000E056E200E066E820E076E7A
:103EA00060EC25F000C0D8F101C0D9F102C0DAF110
:103EB00003C0DBF1C7EC2EF007D10001B005006EA6
:103EC00000C0B0F0060E0101D16F000ED26F00C02D
:103ED000D3F187EC2FF0B0C000F0000E0001B0BFAE
:103EE000FF0E016E36EC2FF029C004F02AC005F059
:103EF0002BC006F02CC007F041EC27F000C029F0E1
:103F000001C02AF002C02BF003C02CF02F0E0101DB
:103F1000D16F000ED26F240ED36F620ED46F000EDD
:103F2000D56F2DC0D6F12EC0D7F1000E046E000E55
:103F3000056E200E066E820E076E60EC25F000C046
:103F4000D8F101C0D9F102C0DAF103C0DBF1C7EC4E
:103F50002EF0BAD00001B105006E00C0B1F0070E1E
:103F60000101D16F000ED26F00C0D3F187EC2FF0AA
:103F7000B1C000F0000E0001B1BFFF0E016E36ECC3
:103F80002FF029C004F02AC005F02BC006F02CC089
:103F900007F041EC27F000C029F001C02AF002C070
:103FA0002BF003C02CF02F0E0101D16F000ED26F49
:103FB000300ED36F620ED46F000ED56F2DC0D6F1C8
:103FC0002EC0D7F1000E046E000E056E200E066E98
:103FD000820E076E60EC25F000C0D8F101C0D9F167
:103FE00002C0DAF103C0DBF1C7EC2EF06DD00001A6
:103FF000B205006E00C0B2F0080E0101D16F000ED4
:10400000D26F00C0D3F187EC2FF0B2C000F0000EE9
:104010000001B2BFFF0E016E36EC2FF029C004F094
:104020002AC005F02BC006F02CC007F041EC27F0A9
:1040300000C029F001C02AF002C02BF003C02CF010
:104040002F0E0101D16F000ED26F3C0ED36F620EA6
:10405000D46F000ED56F2DC0D6F12EC0D7F1000E53
:10406000046E000E056E200E066E820E076E60EC6A
:1040700025F000C0D8F101C0D9F102C0DAF103C0C7
:10408000DBF1C7EC2EF020D00101000E2E1802E16A
:10409000010E2D180101D8B4C3D6000E2E1802E16E
:1040A000020E2D180101D8B408D7000E2E1802E117
:1040B000030E2D180101D8B44DD7000E2E1802E1C1
:1040C000040E2D18010193E0020E0101D16F010EC3
:1040D000D26F2F0ED36F000ED46F7EEC2DF0120036
:1040E000000E296E000E2A6E000E2B6E7F0E2C6EB7
:1040F0002D4A2E2A800E006E800E2E18005C02E1E2
:104100002D50040804E2010E2D6E000E2E6EFCD020
:10411000050E0101D16F000ED26F19EC30F0C3EC27
:104120002FF029C004F02AC005F02BC006F02CC0E7
:1041300007F041EC27F000C029F001C02AF002C0CE
:104140002BF003C02CF02F0E0101D16F000ED26FA7
:10415000B80ED36F610ED46F000ED56F2DC0D6F19F
:104160002EC0D7F1000E046E000E056E200E066EF6
:10417000820E076E60EC25F000C0D8F101C0D9F1C5
:1041800002C0DAF103C0DBF1C7EC2EF0DDD0060E81
:104190000101D16F000ED26F19EC30F0C3EC2FF09B
:1041A00029C004F02AC005F02BC006F02CC007F08F
:1041B00041EC27F000C029F001C02AF002C02BF02A
:1041C00003C02CF02F0E0101D16F000ED26FC40E70
:1041D000D36F610ED46F000ED56F2DC0D6F12EC0F7
:1041E000D7F1000E046E000E056E200E066E820ED4
:1041F000076E60EC25F000C0D8F101C0D9F102C013
:10420000DAF103C0DBF1C7EC2EF09ED0070E0101FE
:10421000D16F000ED26F19EC30F0C3EC2FF029C033
:1042200004F02AC005F02BC006F02CC007F041ECCA
:1042300027F000C029F001C02AF002C02BF003C013
:104240002CF02F0E0101D16F000ED26FD00ED36F64
:10425000610ED46F000ED56F2DC0D6F12EC0D7F1F0
:10426000000E046E000E056E200E066E820E076EA6
:1042700060EC25F000C0D8F101C0D9F102C0DAF13C
:1042800003C0DBF1C7EC2EF05FD0080E0101D16F47
:10429000000ED26F19EC30F0C3EC2FF029C004F0FF
:1042A0002AC005F02BC006F02CC007F041EC27F027
:1042B00000C029F001C02AF002C02BF003C02CF08E
:1042C0002F0E0101D16F000ED26FDC0ED36F610E85
:1042D000D46F000ED56F2DC0D6F12EC0D7F1000ED1
:1042E000046E000E056E200E066E820E076E60ECE8
:1042F00025F000C0D8F101C0D9F102C0DAF103C045
:10430000DBF1C7EC2EF020D00101000E2E1802E1E7
:10431000010E2D180101D8B4FBD6000E2E1802E1B3
:10432000020E2D180101D8B432D7000E2E1802E16A
:10433000030E2D180101D8B469D7000E2E1802E122
:10434000040E2D180101A1E0020E0101D16F010E32
:10435000D26F2F0ED36F000ED46F7EEC2DF01200B3
:10436000E2EC2FF0E2EC2FF0E2EC2FF0C8C100F00D
:10437000010E026E005004E002360290FF0FFBD7E0
:1043800002C01FF0C9C100F0010E016E005004E030
:1043900001360190FF0FFBD701C020F0CAC100F029
:1043A000010E076E005004E007360790FF0FFBD7A1
:1043B00007C021F0CBC100F0010E066E005004E0F2
:1043C00006360690FF0FFBD706C022F0CEC100F0E4
:1043D000010E056E005004E005360590FF0FFBD777
:1043E00005C01EF0CFC100F0010E046E005004E0C5
:1043F00004360490FF0FFBD704C024F0D0C100F0B6
:10440000010E036E005004E003360390FF0FFBD74C
:1044100003C01DF0C6C119F0C7C11AF0CCC11BF012
:10442000CDC11CF019C0E9FF1AC0EAFF1BC0E1FFB3
:104430001CC0E2FF01500210006E0750001206502F
:104440000010026E021C006E0050EF16120E1924AE
:10445000016E01C0E9FF02C000F0001E0050EF161F
:10446000120E015CE96E04500510006E035000123C
:10447000001E0050E716120E1B24016E01C0E1FF62
:104480000050E716120E015CE16E06500710006E38
:104490000050EF120350E71259EC30F01D1C006E73
:1044A0000050E716E2EC2FF01D50E71259EC30F007
:1044B0001D1C006E0050E716E2EC2FF01D50E712B5
:1044C00059EC30F01D1C006E0050E716E2EC2FF0A6
:1044D0002150EF12221C006E0050EF161D50E71203
:1044E00059EC30F01D1C006E0050E716E2EC2FF086
:1044F0001D50E71259EC30F01D1C006E0050E716FD
:10450000211C006E0050EF161F50EF121D50E712D5
:1045100059EC30F01D1C006E0050E716E2EC2FF055
:104520001F1C006E0050EF162250EF121D50E712B4
:1045300059EC30F01D1C006E0050E716221C006E76
:104540000050EF161D50E71259EC30F01D1C006EA4
:104550000050E716E2EC2FF01D50E71259EC30F056
:104560001D1C006E0050E7162250EF121D50E7127E
:1045700059EC30F01D1C006E0050E716E2EC2FF0F5
:10458000221C006E0050EF161D50E71259EC30F05F
:104590001D1C006E0050E71621502210006E2050A6
:1045A00000121F5000120050EF121D50E71259EC7C
:1045B00030F01D1C006E0050E716E2EC2FF0010EEB
:1045C000236E120000010CB025EF23F00CA2CDEFFA
:1045D00023F00E6A000E02643CEF23F0F00E02148A
:1045E000D8A407EF23F0023A01380F0B0226013856
:1045F000F00B016E00380F0B01260038F00B006E37
:1046000008380F0B00260838F00B086E0E84D8907F
:1046100002BE20EF23F008360036013602360E2A9D
:1046200002BE20EF23F008360036013602360E2A8D
:1046300002BE20EF23F008360036013602360E2A7D
:104640000E500364C1EF23F0035E0BBC08AEC7EF4E
:1046500023F0D880800E08640030000E0022012272
:104660000222D8A0C7EF23F0023201320032034AFF
:10467000CDEF23F0C7EF23F001C002F000C001F03E
:1046800008C000F0086A000E0E86026473EF23F083
:10469000F00E0214D8A45BEF23F0023A01380F0B9E
:1046A00002260138F00B016E00380F0B012600388E
:1046B000F00B006E0E84D89002BE20EF23F000367F
:1046C000013602360E2A02BE20EF23F000360136F4
:1046D00002360E2A02BE20EF23F0003601360236E3
:1046E0000E2A20EF23F001C002F000C001F0006AA2
:1046F000000E0E960E880264A0EF23F0F00E021456
:10470000D8A48BEF23F0023A01380F0B02260138B0
:10471000F00B016E0E84D89002BE20EF23F001361C
:1047200002360E2A02BE20EF23F0013602360E2A90
:1047300002BE20EF23F0013602360E2A20EF23F0CE
:1047400001C002F0016A000E0E860264D3EF23F06E
:10475000F00E0214D8A4AFEF23F0023A0E84D890E2
:1047600002BE20EF23F002360E2A02BE20EF23F015
:1047700002360E2A02BE20EF23F002360E2A20EF68
:1047800023F0010E0C6EF1EC2FF0D7EF23F0020EA8
:104790000C6E4AEC30F0D7EF23F0040E0C6EFFECF9
:1047A0002FF0D7EF23F0080E0C6E35EC30F012002E
:1047B000200E0101B66FB76B2E0EB86FB96B010EEC
:1047C0007919006E00C079F100520BE0020ED16F32
:1047D000100ED26FB60ED36F010ED46F7EEC2DF09B
:1047E0000AD0020ED16F100ED26FB80ED36F010E29
:1047F000D46F7EEC2DF0576B586B800E5819006EFD
:10480000800E005C02E1080E575DD8B09FD00051C9
:10481000000A0CE1F80E8C16EAEC2BF000C059F1FE
:1048200001C05AF102C05BF103C05CF1010100510B
:10483000010A0BE18C8096EC2BF000C05DF101C009
:104840005EF102C05FF103C060F101010051020A94
:1048500012E1F80E8C14006E00C08CFF020E0010E6
:104860008C6E92EC2CF000C061F101C062F102C0CC
:1048700063F103C064F101010051030A0CE1030E6E
:104880008C123EEC2CF000C065F101C066F102C054
:1048900067F103C068F101010051040A12E1F80E4A
:1048A0008C14006E00C08CFF040E00108C6E9AEC0D
:1048B0002AF000C069F101C06AF102C06BF103C0C7
:1048C0006CF101010051050A0CE1050E8C1246EC59
:1048D0002AF000C06DF101C06EF102C06FF103C09B
:1048E00070F101010051060A12E1F80E8C14006EFD
:1048F00000C08CFF060E00108C6E42EC2BF000C046
:1049000071F101C072F102C073F103C074F10101D1
:104910000051070A0CE1070E8C12EEEC2AF000C0E1
:1049200075F101C076F102C077F103C078F144EC73
:1049300030F00101002B800E070A006E800E001976
:10494000005CD8A0006B574B582B57D712000101C1
:10495000576B586B800E5819006E800E005C02E198
:10496000280E575DD8B0ABD0046A8CB8042A010E6B
:104970000418006E000E00B0100E8C18100B8C1A6C
:104980000051000A0CE1F80E8C16EAEC2BF000C086
:1049900059F101C05AF102C05BF103C05CF10101A1
:1049A0000051010A0BE18C8096EC2BF000C05DF108
:1049B00001C05EF102C05FF103C060F1010100516E
:1049C000020A12E1F80E8C14006E00C08CFF020E79
:1049D00000108C6E92EC2CF000C061F101C062F10D
:1049E00002C063F103C064F101010051030A0CE14C
:1049F000030E8C123EEC2CF000C065F101C066F194
:104A000002C067F103C068F101010051040A12E11C
:104A1000F80E8C14006E00C08CFF040E00108C6E1B
:104A20009AEC2AF000C069F101C06AF102C06BF192
:104A300003C06CF101010051050A0CE1050E8C1256
:104A400046EC2AF000C06DF101C06EF102C06FF1BA
:104A500003C070F101010051060A12E1F80E8C1436
:104A6000006E00C08CFF060E00108C6E42EC2BF026
:104A700000C071F101C072F102C073F103C074F1A2
:104A800001010051070A0CE1070E8C12EEEC2AF02E
:104A900000C075F101C076F102C077F103C078F172
:104AA00044EC30F00101002B800E070A006E800EEE
:104AB0000019005CD8A0006B574B582B4BD7120045
:104AC0000001086A096A0750D8B4F7EF25F00350CF
:104AD000D8B4FCEF25F0025006180A6E028E068E3E
:104AE0000E6A02C008F001C00CF000C00DF00450C6
:104AF0000D5E0550D8A0053C0C5E0650D8A0063CC3
:104B0000085E086A0C6A0D6AD8A08EEF25F0D8906E
:104B10000232013200320832010E0E6E0750035E7F
:104B2000D8A09BEF25F07E0E0E240326D8B001EF0F
:104B300026F0A1EF25F07E0E0E240326D8A006EF66
:104B400026F0180E0B6E0D360C3608360036013680
:104B500002360E360450005E0550D8A0053C015EBA
:104B60000650D8A0063C025E06340E120EA0BCEF22
:104B700025F00D80C7EF25F0045000260550D8B071
:104B8000053C01260650D8B0062802260D900B2EB3
:104B9000A3EF25F0EDEF25F0D89000360136023670
:104BA0000E360450005E0550D8A0053C015E06504C
:104BB000D8A0063C025E06340E10010B0D26D8B0BC
:104BC0000C2AD8B4082AD8A4EDEF25F008320C320C
:104BD0000D32032AD8B401EF26F00AAE089E085021
:104BE000026E0C50016E0D50006E09EF26F0010EA2
:104BF00054EC30F009EF26F0020E35EC30F009EFFE
:104C000026F0040EFFEC2FF009EF26F0080EF1EC71
:104C10002FF0120000010B6A0C6A0A6A086A03503E
:104C2000D8B493EF26F0028E9E0E035E03BE1EEFF5
:104C300026F0D8B41EEF26F083EF26F0036C080EA2
:104C4000035CD8A050EF26F0036E083600C008F0D1
:104C500001C000F002C001F0026A080E035CD8A097
:104C600050EF26F0036E083600C008F001C000F0D7
:104C7000016A080E035CD8A050EF26F0036E0836D8
:104C800000C008F0006A080E035CD8A050EF26F0C0
:104C9000036E0836086A0350D8A4D8905CEF26F05B
:104CA0000350D8B45CEF26F0D890023201320032C3
:104CB0000832032E54EF26F00BBC08A06DEF26F04F
:104CC000D8A06DEF26F0082AD8B4002AD8B4012A5B
:104CD000D8B4022A02BE97EF26F00AAE93EF26F070
:104CE000021E011E001E081E082AD8B4002AD8B4CD
:104CF000012AD8B4022A93EF26F0026A016A006AF8
:104D0000086A93EF26F00B800BAE9DEF26F0026A47
:104D10000AAE9DEF26F0026E016E006E086E0A3636
:104D200002329DEF26F0000E0C6A9EEF26F0010E77
:104D30000C6ED3EC2FF09EEF26F0FF0E0250036EA8
:104D40000150026E0050016E0850006E120000010A
:104D50000B6A0C6A086A0350D8B42CEF27F002C023
:104D60000AF0028E9E0E035E03AE1CEF27F0036C6A
:104D7000080E035CD8A0E9EF26F0036E083600C0E9
:104D800008F001C000F002C001F0026A080E035CE6
:104D9000D8A0E9EF26F0036E083600C008F001C085
:104DA00000F0016A080E035CD8A0E9EF26F0036E5C
:104DB000083600C008F0006A080E035CD8A0E9EFCE
:104DC00026F0036E0836086A0350D8A4D890F5EF91
:104DD00026F00350D8B4F5EF26F0D8900232013215
:104DE00000320832032EEDEF26F00BBC08A006EFD0
:104DF00027F0D8A006EF27F0082AD8B4002AD8B4A4
:104E0000012AD8B4022A02BE30EF27F00AAE2CEFF6
:104E100027F0021E011E001E081E082AD8B4002A10
:104E2000D8B4012AD8B4022A2CEF27F0026A016A0A
:104E3000006A086A2CEF27F00B800BAE37EF27F0E3
:104E4000026A0AAE37EF27F0026E016E006E086E3E
:104E50000A36023237EF27F00C6A000E38EF27F0DF
:104E6000010E0C6E000ED3EC2FF038EF27F0FF0E82
:104E70000250036E0150026E0050016E0850006E29
:104E800012000001086A096A000E07620364C7EF96
:104E900027F0025006180A6E075003267E0ED8A08F
:104EA00058EF27F0035ED8B0CCEF27F05CEF27F087
:104EB000035ED8A0D1EF27F0028E068E02C00EF05E
:104EC00001C00BF000C00DF000500402F4CF0CF054
:104ED00001500502F4CF00F0F3CF08F00402F350C4
:104EE0000C26F4500822000E00220D500502F3504B
:104EF0000C26F4500822000E002202500402F35047
:104F00000826F450002202500502016A000E012218
:104F1000F3500026F45001220D500602F3500826EB
:104F2000F4500022026A000E012202220B500602F7
:104F3000F3500026F4500122000E02220E50060209
:104F4000F3500126F450022202BEAFEF27F00836DC
:104F50000036013602360306D8B4D1EF27F0C2EF8F
:104F600027F0D880800E08640030000E0022012255
:104F70000222D8A0C2EF27F0023201320032034AE7
:104F8000CCEF27F00AAE029E000ED4EF27F0010E00
:104F900035EC30F0D4EF27F0020EFFEC2FF0D4EF19
:104FA00027F0040EF1EC2FF0120019C0E9FF1AC02F
:104FB000EAFF1BC0E1FF1CC0E2FF1D1C006E005099
:104FC000E7161E1C006E0050E71620501F10006EE2
:104FD0002150001222500012001E0050EF16020154
:104FE00009AF02D01F50EF1209AD02D02050EF12CE
:104FF00009AB02D02150EF1209A902D02250EF12C2
:10500000235205E01E1C006E0050E71603D002017B
:105010001E50E7121D50E71259EC30F01D1C006EB7
:105020000050E7161E1C006E0050E71620501F109F
:10503000006E2150001222500012001E0050EF1688
:10504000020109A702D01F50EF1209A502D020507B
:10505000EF1209A302D02150EF1209A102D0225071
:10506000EF12235205E01E1C006E0050E71603D01D
:1050700002011E50E71202011D50E71259EC30F0F8
:105080001D1C006E0050E716235203E0E2EC2FF0E7
:1050900002D03DEC30F01200780E01017B6F440E1F
:1050A0007C6F410E7D6F540E7E6F410E7F6F780EC8
:1050B000806F780E816F780E826F430E836F530E70
:1050C000846F560E856F866B000E876F000E886F9B
:1050D000000E006F000E896F000E7A6F000E156EC5
:1050E000000E166E000E176E000E186E000E8A6F00
:1050F000000E8B6F000E8C6F000E8D6F000E000186
:10510000FF6F000E01018E6F000E8F6F000E906F0B
:10511000000E916F000E796F000E256E000E266E48
:10512000000E276E000E286E340E926F2D0E936FB8
:10513000430E946F680E956F610E966F6E0E976FAB
:105140006E0E986F650E996F6C0E9A6F200E9B6FA6
:10515000500E9C6F740E9D6F310E9E6F300E9F6FC0
:10516000300EA06FA16B920E556F010E566F000EA0
:105170002D6E000E2E6E120000010A6A0350D8A494
:105180000A800750D8A40A820A50D8B420EF29F028
:10519000030AD8B4D9EF28F00AB0D4EF28F006AE4D
:1051A0001EEF29F01CEF29F002AE1CEF29F01EEFD4
:1051B00029F00250800B0A6E029E0650800B069E5C
:1051C0000A18D8B4EAEF28F00A50D8B41CEF29F036
:1051D0001EEF29F00750035CD8B4F4EF28F0D8A0F4
:1051E00010EF29F016EF29F00650025CD8B4FEEF5C
:1051F00028F0D8A010EF29F016EF29F00550015C37
:10520000D8B408EF29F0D8A010EF29F016EF29F054
:105210000450005CD8B420EF29F0D8B016EF29F084
:105220000A52D8B41EEF29F01CEF29F00A52D8B464
:105230001CEF29F01EEF29F0D8801200D890120040
:10524000D880D8841200120000010D6A096A086A29
:1052500001500010D8B4000C015005180A6E0ABEA7
:105260000D1E0B6A05AE3AEF29F0041E051E042A36
:10527000D8B4052A01AE42EF29F0001E011E002A13
:10528000D8B4012A015005100A6E0ABE5AEF29F05F
:105290006DEC2EF00BB071EF29F00DAE000C001E7E
:1052A000011E002AD8B4012A081E091E082AD8B4F3
:1052B000092A000C05AE6CEF29F001BE68EF29F059
:1052C0000150096E0050086E016A006A4DEF29F026
:1052D000016A006A002A000C011E001E0B2A48EF1A
:1052E00029F0082AD8B4092A0450085CD8A44DEF44
:1052F00029F00550095CD8A44DEF29F0096A086A25
:10530000002AD8B4012A01AE4DEF29F00000FF0CAD
:1053100012000101D26BD36BD46BD56B839AD16B26
:10532000200ED15D29E2D2C108F0D3C109F0D4C169
:105330000AF0D5C10BF00836089009360A360B364C
:1053400008C0D2F109C0D3F10AC0D4F10BC0D5F125
:10535000838E046A83BC042A04500810D26F09C0EB
:10536000D3F10AC0D4F10BC0D5F1000ED313D4137E
:10537000D513839ED12BD4D7838AFF0ED215046E0A
:10538000FF0ED315056EFF0ED415066E1F0ED51534
:10539000076E04C0D2F105C0D3F106C0D4F107C036
:1053A000D5F107A805D0006A016A026A036A1200F3
:1053B000D3C100F0D4C101F0D5C102F0000ED5BFB9
:1053C000FF0E036E00C0D2F101C0D3F102C0D4F1D0
:1053D00003C0D5F1120000010D6A086A0050D8B46C
:1053E000000C04180A6E0ABE0D1E0B6A04AEFBEF19
:1053F00029F0041E042A00A000EF2AF0001E002A53
:10540000005004100A6E0ABE27EF2AF00450085E0E
:10541000003600340836045008260036060E0C6E9E
:1054200000340836045000B0085E00A0082600369C
:105430000C2E10EF2AF000A008260BB039EF2AF04E
:105440000DAE000C001E002A081E082A000C04AE37
:1054500035EF2AF000BE32EF2AF00050086E006AE5
:1054600020EF2AF0006A002A000C001E0B2A06EF2B
:105470002AF0082A0450085CD8A420EF2AF0086A11
:10548000002A00AE20EF2AF0FF0C12001DC119F116
:105490001EC11AF11FC11BF120C11CF121C11DF158
:1054A00022C11EF123C11FF124C120F125C121F128
:1054B00026C122F127C123F128C124F129C125F1F8
:1054C0002AC126F12BC127F12CC128F189EC29F042
:1054D00000C029F101C02AF102C02BF103C02CF158
:1054E000010125510026265101222751022228516F
:1054F000032221510026225101222351022224514C
:1055000003221D5100261E5101221F51022220514B
:105510000322195100261A5101221B5102221C514B
:105520000322050E046E000E056E066E076E10EC6B
:105530001CF0120009C105F10AC106F10BC107F107
:105540000CC108F10DC109F10EC10AF10FC10BF137
:1055500010C10CF111C10DF112C10EF113C10FF107
:1055600014C110F115C111F116C112F117C113F1D7
:1055700018C114F189EC29F000C015F101C016F131
:1055800002C017F103C018F1010111510026125198
:10559000012213510222145103220D5100260E51F3
:1055A00001220F51022210510322095100260A51F3
:1055B00001220B5102220C510322055100260651F3
:1055C00001220751022208510322050E046E000E2B
:1055D000056E066E076E10EC1CF0120045C141F11D
:1055E00046C142F147C143F148C144F149C145F1C7
:1055F0004AC146F14BC147F14CC148F14DC149F197
:105600004EC14AF14FC14BF150C14CF151C14DF166
:1056100052C14EF153C14FF154C150F189EC29F000
:1056200000C051F101C052F102C053F103C054F166
:1056300001014D5100264E5101224F51022250517D
:105640000322495100264A5101224B5102224C515A
:10565000032245510026465101224751022248515A
:10566000032241510026425101224351022244515A
:105670000322050E046E000E056E066E076E10EC1A
:105680001CF0120031C12DF132C12EF133C12FF1C6
:1056900034C130F135C131F136C132F137C133F1A6
:1056A00038C134F139C135F13AC136F13BC137F176
:1056B0003CC138F13DC139F13EC13AF13FC13BF146
:1056C00040C13CF189EC29F000C03DF101C03EF140
:1056D00002C03FF103C040F10101395100263A51A7
:1056E00001223B5102223C51032235510026365102
:1056F0000122375102223851032231510026325102
:10570000012233510222345103222D5100262E5101
:1057100001222F51022230510322050E046E000E89
:10572000056E066E076E10EC1CF01200CBC0C7F0C1
:10573000CCC0C8F0CDC0C9F0CEC0CAF0CFC0CBF04D
:10574000D0C0CCF0D1C0CDF0D2C0CEF0D3C0CFF01D
:10575000D4C0D0F0D5C0D1F0D6C0D2F0D7C0D3F0ED
:10576000D8C0D4F0D9C0D5F0DAC0D6F089EC29F091
:1057700000C0D7F001C0D8F002C0D9F003C0DAF001
:105780000001D3510026D4510122D5510222D65115
:105790000322CF510026D0510122D1510222D251F1
:1057A0000322CB510026CC510122CD510222CE51F1
:1057B0000322C7510026C8510122C9510222CA51F1
:1057C0000322050E046E000E056E066E076E10ECC9
:1057D0001CF01200B7C0B3F0B8C0B4F0B9C0B5F057
:1057E000BAC0B6F0BBC0B7F0BCC0B8F0BDC0B9F02D
:1057F000BEC0BAF0BFC0BBF0C0C0BCF0C1C0BDF0FD
:10580000C2C0BEF0C3C0BFF0C4C0C0F0C5C0C1F0CC
:10581000C6C0C2F089EC29F000C0C3F001C0C4F0DA
:1058200002C0C5F003C0C6F00001BF510026C05140
:105830000122C1510222C2510322BB510026BC5198
:105840000122BD510222BE510322B7510026B85198
:105850000122B9510222BA510322B3510026B45198
:105860000122B5510222B6510322050E046E000E2C
:10587000056E066E076E10EC1CF01200F3C0EFF020
:10588000F4C0F0F0F5C0F1F0F6C0F2F0F7C0F3F0BC
:10589000F8C0F4F0F9C0F5F0FAC0F6F0FBC0F7F08C
:1058A000FCC0F8F0FDC0F9F0FEC0FAF001C1FBF059
:1058B00002C1FCF003C1FDF004C1FEF089EC29F047
:1058C00000C001F101C002F102C003F103C004F104
:1058D0000001FB510026FC510122FD510222FE5124
:1058E0000322F7510026F8510122F9510222FA5100
:1058F0000322F3510026F4510122F5510222F65100
:105900000322EF510026F0510122F1510222F251FF
:105910000322050E046E000E056E066E076E10EC77
:105920001CF01200DFC0DBF0E0C0DCF0E1C0DDF015
:10593000E2C0DEF0E3C0DFF0E4C0E0F0E5C0E1F09B
:10594000E6C0E2F0E7C0E3F0E8C0E4F0E9C0E5F06B
:10595000EAC0E6F0EBC0E7F0ECC0E8F0EDC0E9F03B
:10596000EEC0EAF089EC29F000C0EBF001C0ECF0E9
:1059700002C0EDF003C0EEF00001E7510026E8514F
:105980000122E9510222EA510322E3510026E451A7
:105990000122E5510222E6510322DF510026E051A7
:1059A0000122E1510222E2510322DB510026DC51A7
:1059B0000122DD510222DE510322050E046E000E8B
:1059C000056E066E076E10EC1CF01200200E010131
:1059D000B66F200EB76F540EB86F680EB96F650EB4
:1059E000BA6F720EBB6F6D0EBC6F6F0EBD6F6D0E1A
:1059F000BE6F650EBF6F740EC06F650EC16F720E05
:105A0000C26FC36B810EC66F0F0EC76F070EC86FD4
:105A1000060EC96F050ECA6F040ECB6F810ECC6FD8
:105A20000F0ECD6F020ECE6F010ECF6F030ED06F33
:105A3000B0EC21F00C0E0201096FD5EC27F0010E3D
:105A40000101D16F010ED26F55C1D3F156C1D4F10E
:105A50007EEC2DF0020ED16F010ED26FB60ED36F19
:105A6000010ED46F7EEC2DF012004CEC28F0400EAD
:105A7000D36E836A400E956E0A0EC16EFF0E926E53
:105A8000070E9612FF0E846E936AFF0E816E930EC0
:105A9000946EFF0E826E8A8A1F0ECD6ECF6ACE6A1A
:105AA000AF0ED56ED59ED76AD66AC00EF26EF18E55
:105AB0009E90E6EC2CF0B66BB76BB86B010EB96F2D
:105AC00070EC2FF08C988C969D8001EC2EF00001EC
:105AD000AF6BEDEC2EF00001FF5303E012EC2FF062
:105AE000FAD7A7EC24F0010E0201096FD5EC27F0DC
:105AF000D8EC23F0DBEC11F0FBD7FFD710D0800EF1
:105B00000101D16F1AD0C00ED16F17D0940ED16F92
:105B100014D0D40ED16F11D0800ED16F0ED00101F0
:105B2000D151010AECE0D151020AEDE0D151030A52
:105B3000EDE0D151040AEDE0EFD7D205006ED1516E
:105B4000002600C0D1F100C009F2D5EC27F0236A8D
:105B50000101D56BD551D325E96E000ED421EA6E33
:105B6000EECF00F000520DE0D551D325E96E000EC6
:105B7000D421EA6EEECFE0F12DEC30F00101D52B0F
:105B8000E9D7010E236E120000010C6A0E6A025062
:105B9000D8A4DEEF2DF001C002F000C001F0006AD1
:105BA0000E860250D8A4DEEF2DF001C002F0016A8B
:105BB0000E960E880250D8B4F0EF2DF00E50035E12
:105BC000D8A4D8A0F6EF2DF0D89002BEFCEF2DF0AF
:105BD000003601360236032EE5EF2DF0F6EF2DF0FC
:105BE000010E0C6E35EC30F000EF2EF0020E0C6E54
:105BF000F1EC2FF000EF2EF0040E0C6E4AEC30F0BA
:105C00001200430E0101B66F610EB76F6C0EB86FD4
:105C1000690EB96F620EBA6F720EBB6F610EBC6F08
:105C2000740EBD6F650EBE6F200EBF6F4D0EC06F40
:105C30006F0EC16F640EC26F650EC36FC46B016AD5
:105C400084B4012A0150000A13E1010E0001FF6F24
:105C5000010E0201096FD5EC27F0010E0101D16F91
:105C6000010ED26FB60ED36F010ED46F7EEC2DF005
:105C70001200000100500402F4CF09F0F3CF08F045
:105C800001500502F4CF0BF0F3CF0AF000500502EB
:105C9000F3500926F4500A22E86A0B22015004024C
:105CA000F3500926F4500A22E86A0B2205AE5DEF94
:105CB0002EF000500A5C01500B5801AE64EF2EF03C
:105CC00004500A5C05500B5808C000F009C001F0F0
:105CD0000AC002F00BC003F01200000101340836C4
:105CE00009360450085E0550D8A0053C095E003610
:105CF00001360F0E0C6E013408360936045000A030
:105D000089EF2EF0085E0550D8A0053C095E8EEFA5
:105D10002EF008260550D8B0053C0926003601367D
:105D20000C2E7BEF2EF000B09CEF2EF004500826D6
:105D30000550D8B0053C092600001200256A016A0A
:105D400084B4012A0150000A07E12650000A04E148
:105D5000010E266E010E256E016A84B2012A0150E1
:105D6000000A07E12750000A04E1010E276E020E27
:105D7000256E010E8414016E0150000A07E12850BF
:105D8000000A04E1010E286E030E256E1200D60EE5
:105D90000101DE6F010EDF6FD1C1E0F1D2C1E1F18F
:105DA000D3C1E2F1D4C1E3F1D5C1E4F1DE0EE56F78
:105DB000010EE66F20EC00F000C0DCF101C0DDF167
:105DC00000500101D125E16E0150D221E26EE66A58
:105DD000DCC100F0DDC101F01200050E0101D16F40
:105DE000000ED26F19EC30F000C0AFF0060E0101CA
:105DF000D16F000ED26F19EC30F000C0B0F0070E7A
:105E00000101D16F000ED26F19EC30F000C0B1F07B
:105E1000080E0101D16F000ED26F19EC30F000C0F6
:105E2000B2F012000A0E0B6EFF0E0A6E0B2E01D09E
:105E300003D00A2EFED7FAD7B60E0A6E0A2EFED768
:105E40009EEC2EF023EC30F02550010A02E170ECBC
:105E500020F001012550020A02E19AEC1DF0010137
:105E60002550030A02E107EC1FF01200000100C0F8
:105E700008F00150006E016A026A036A0B6A0C6A3C
:105E8000016A026A036A960E036E0A6A00AE4FEF59
:105E90002FF0081E001E082AD8B4002A0A8E00C05F
:105EA00001F008C000F0086A026AC4EC2DF012008C
:105EB000000103500718D8A46DEF2FF00250061808
:105EC000D8A46DEF2FF001500518D8A46DEF2FF076
:105ED00000500418D8B4D8841200D89412001200CC
:105EE000949A94969488C66A0101B651C612B85124
:105EF000C612B751C712B85305E0B951000AD8B459
:105F0000C78C03D0B953D8A4C78CC68A1200A6A2E6
:105F100002D00000FCD7A69CD2C1AAFFD1C1A9FF24
:105F2000D3C1A8FFA69EA684F29E550EA76EAA0E08
:105F3000A76EA682F28EA694120000010050086E91
:105F40000150006E0250016E0350026E036A0B6A2C
:105F50000C6A9E0E036E0A6A020E0C6EE2EC22F0D0
:105F600012000001086B080E0C6E00340836045055
:105F7000085ED8B0BEEF2FF00826D89000360C2E61
:105F8000B5EF2FF01200000100C008F00B6A0C6A98
:105F90009E0E036E0A6A026A016A006A020E0C6EA5
:105FA000E2EC22F0120000010B800BAEE0EF2FF0CC
:105FB000026A0AAEFF0E026E016E006E0A360232EF
:105FC000FF0E1200020E0B6EFF0E0A6E0B2E01D09A
:105FD00003D00A2EFED7FAD7C70E0A6E0A2EFED7B6
:105FE000120000010B840BAEFDEF2FF0010E036ECB
:105FF000026A016A006A0A360232FF0E12000001CC
:106000000B820BAE0AEF30F003680268016800688B
:106010000A360232FF0E120002010951390807E365
:10602000300E095D04E3010E006E18EF30F0006AD7
:106030001200A69CD2C1AAFFD1C1A9FFA69EA6802C
:10604000A8CF00F0120084B4266A84B2276A010E39
:106050008414006ED8A4286A1200236AE0C109F2F1
:10606000D5EC27F0010E236E12000001026A016ACE
:10607000006A086A036A000E1200030E0A6E0A2EF6
:10608000FED7000000001200839E839A83BCFED7D7
:10609000838A120000010AAE029E000E1200000167
:1060A000067E69EC18F0120000010B6A0B86FF0EE9
:1060B000120012000000007FCDCC4C7B0AD7237861
:1060C0006F12037517B75171ACC5276EBD37066BDC
:1060D00095BF566777CC2B645F700961FFE65B5D07
:1060E00008E53C3C6042221B0000007F000020824B
:1060F0000000488500007A8800401C8C0050438FC7
:10610000002474928096189620BC3E99286B6E9C51
:10611000F90215A0EC782DC1CAF249E20100000095
:106120000A00000064000000E803000010270000DF
:10613000A086010040420F008096980000E1F5051E
:1061400000CA9A3B0100000010000000000100009E
:10615000001000000000010000001000000000011D
:1061600000000010010000000800000040000000D6
:106170000002000000100000008000000000040089
:1061800000002000000000010000000800000040A6
:10619000000000003031323334353637383941426F
:1061A0004344454600FF30313233343536373839D1
:1061B00061626364656600FF434825642025312ED3
:1061C00031662000434825642025312E31662000A9
:1061D000434825642025312E31662000434825643C
:1061E0002025312E31662000434825642025312E9C
:1061F00031662000434825642025312E3166200079
:10620000434825642025312E31662000434825640B
:106210002025312E31662000434825642025312E6B
:1062200031662000434825642025312E3166200048
:10623000434825642025312E3166200043482564DB
:106240002025312E31662000313D252E3166430058
:10625000333D252E31664300323D252E3166430005
:10626000343D252E31664300FFFFFFFFFFFFFFFF98
:020000040030CA
:0E000000FFF8FFFEFFFFBBFFFFFFFFFFFFFF4C
:00000001FF
